:020000040800F2
:10C80000C819002045C9000811DB000803D9000839
:10C810000DDB0008EDD300087BEA000800000000F3
:10C8200000000000000000000000000003E000081D
:10C83000F1D3000800000000D9DB000835E1000852
:10C840005FC900085FC900085FC900085FC9000828
:10C850005FC900085FC90008F5D3000821D40008AB
:10C860004DD400085FC900085FC900085FC900080F
:10C870005FC900085FC900085FC900085FC90008F8
:10C880005FC900085FC900085FC900085FC90008E8
:10C890005FC900085FC900085FC9000879D40008B3
:10C8A0005FC90008D9E300085FC900085FC9000834
:10C8B0003DE4000801E500085FC900085FC9000801
:10C8C0005FC900085FC900085FC900085FC90008A8
:10C8D0005FC90008E1E700085FC9000869E80008CF
:10C8E0005FC900085FC900085FC900085FC9000888
:10C8F0005FC900085FC900085FC900085FC9000878
:10C900005FC900085FC900085FC900085FC9000867
:10C910005FC900085FC900085FC900085FC9000857
:10C920005FC900085FC900085FC900085FC9000847
:10C93000DFF80CD000F010FC0048004795FA000822
:10C94000C81900200648804706480047FEE7FEE772
:10C95000FEE7FEE7FEE7FEE7FEE7FEE7FEE7FEE7AF
:10C9600039E1000831C9000840EA01039B0703D000
:10C9700009E008C9121F08C0042AFAD203E011F81E
:10C98000013B00F8013B521EF9D27047D2B201E0E0
:10C9900000F8012B491EFBD270470022F6E710B5C4
:10C9A00013460A4604461946FFF7F0FF204610BD1D
:10C9B000421C10F8011B0029FBD1801A704730B5CA
:10C9C00004460020034600E05B1C934203D2E05C77
:10C9D000CD5C401BF8D030BDF0B480EA0102D40F2A
:10C9E0004200B2EB410F02D20246084611464A000D
:10C9F00042D0C30DDDB2C1F3C752AD1A202D35DAD6
:10CA0000C1F3160141F4000204B15242C5F12006FF
:10CA100002FA06F12A411044B3EBD05F23D0C4B12F
:10CA2000012DA0EBC35009DCF0BC4FF0004202EA3C
:10CA3000C352DBB200F5000000F02CBA400000F158
:10CA4000807000EBC350A0F1807040EAD1704900C3
:10CA500009E0490841EAC071A0EBC35000F50000AD
:10CA6000400800EBC350F0BC00F00BBA6142012259
:10CA700002EB4101001BF6E7F0BC704781F000417A
:10CA8000AAE780F00040A7E780EA010210B502F0B3
:10CA90000043400022D04A001FD0010E01EB12617A
:10CAA000C0F35600C2F3560240F4000042F4000204
:10CAB000A0FB022000047F39140400D0401C50EA7F
:10CAC000124001D44000491EC2B20C0604EBD01043
:10CAD000401C4008802A02D003E0002010BD20F056
:10CAE0000100002900DA0020184310BD30B480EAAC
:10CAF000010202F0004530F0004221F0004013D066
:10CB000090B1C30DD40DC2F31601C0F31600E41AA0
:10CB100041F4000140F400027D34914201D3641CD1
:10CB200000E04900002C02DA30BC002070474FF4CE
:10CB300000000023914201D3891A034340084FEAC1
:10CB40004101F7D151B1914202D14FF0004105E0CE
:10CB500002D24FF0010101E06FF0010103EBC4507C
:10CB6000284430BC00F08DB92DE9FE4F81EA030462
:10CB700004F0004421F0004100944FF0000B23F03A
:10CB8000004350EA01045ED052EA03045BD0C3F3D1
:10CB90000A54C1F30A552C44A4F2F3340194A0FBC7
:10CBA0000254C1F3130141F48011C3F3130343F49E
:10CBB000801301FB024400FB034E840A970A44EAF7
:10CBC000815447EA8357A4FB076802958D0A05FB49
:10CBD00007854FEA932C04FB0C542705029D4FEA6E
:10CBE000065847EA1637B5EB08056EEB070C870EBB
:10CBF000920E47EA811742EA8312A7FB0201B6EBC5
:10CC00000B0164EB00042B0D43EA0C335E1844EB7C
:10CC10001C50DA465146E7FB0201C5F313044FEA04
:10CC20000B3343EA14534FEA0432019C43EA0603F0
:10CC3000A4F10C040294009CCDE900B400F067F963
:10CC400003B0BDE8F08F00200146F9E72DE9F04D73
:10CC500081EA030404F0004B21F0004514464FF034
:10CC6000000A23F0004150EA050220D054EA0102F4
:10CC70001DD0C5F30A570246C5F31303C1F31300D1
:10CC8000C1F30A5640F4801543F48013A7EB06085D
:10CC9000101BD64608F2FD3873EB050002D308F1ED
:10CCA000010801E092185B41B8F1000F03DA00209F
:10CCB0000146BDE8F08D00204FF480110646844601
:10CCC0000EE0171B73EB050705D3121B63EB05037F
:10CCD00006434CEA010C49084FEA300092185B41C8
:10CCE00050EA0107EDD152EA030012D082EA0400B3
:10CCF00083EA0501084305D0101BAB4106D201228F
:10CD0000002306E000224FF0004302E06FF0010232
:10CD100053101AEB06004CEB085110EB0A0041EBE4
:10CD20000B01BDE8F04D00F0E3B896230022114658
:10CD300000F0B0B80EB540F2334102910021CDE9C8
:10CD400000110A460B4600F0E2F803B000BD20F0E7
:10CD50000040C10DC0F3160040F400007F2901DA45
:10CD600000207047962903DCC1F19601C840704746
:10CD700096398840704700F0004230F000400AD0F9
:10CD8000C10D01F56071C0F3160042EA0151C208FD
:10CD900040071143704700200146704701F00043EF
:10CDA00030B421F0004150EA010206D00A0DA2F58C
:10CDB0006072C1F31301002A02DC30BC002070470E
:10CDC000440F44EAC104C100E01830BC00EBC2507B
:10CDD00000F057B830B50B46014600202022012450
:10CDE00009E021FA02F59D4205D303FA02F5491B39
:10CDF00004FA02F52844151EA2F10102F1DC30BD4F
:10CE00002DE9F05F0546002092469B46884606467F
:10CE1000814640241BE0284641464746224600F012
:10CE200020F853465A46C01A914110D3114618466D
:10CE3000224600F0A3F92D1A67EB01084F4622465F
:10CE40000120002100F09AF917EB00094E41201E45
:10CE5000A4F10104DFDC484631462A464346BDE8DA
:10CE6000F09F202A04DB203A21FA02F000217047CB
:10CE700021FA02F3D040C2F1200291400843194642
:10CE800070470029A8BF7047401C490008BF20F028
:10CE90000100704710B4B0FA80FC00FA0CF050EAC0
:10CEA000010404BF10BC704749B1CCF1200421FA41
:10CEB00004F411FA0CF118BF012121430843A3EB3C
:10CEC0000C01CB1D4FEA00614FEA102042BF002049
:10CED00010BC704700EBC35010440029A4BF10BC25
:10CEE0007047401C490008BF20F0010010BC70478B
:10CEF00010B5141E73F1000408DA401C41F1000162
:10CF000092185B411A4301D120F0010010BD2DE9B8
:10CF1000F04D92469B4611B1B1FA81F202E0B0FAAF
:10CF200080F22032904600F029F904460F4640EA8C
:10CF30000A0041EA0B0153465A46084313D01146F2
:10CF400053EA010019D0C8F140025046FFF789FFAB
:10CF500005460E4650465946424600F00FF9084332
:10CF600005D0012004E020463946BDE8F08D0020C0
:10CF7000054346EAE0762C4337430A986305E40A02
:10CF8000A0EB08000022FD0A44EA47540A3002D50B
:10CF900000200146E9E7010510196941DDE908456E
:10CFA00000196941BDE8F04DA2E72DE9FE4F80462A
:10CFB00081EA0300C00F0C46009021F0004123F0ED
:10CFC0000045B8EB0200A94105D2404621469046F3
:10CFD0001C460B46024623F00040104347D0270D65
:10CFE000C7F30A00C3F30A510290401A0190402887
:10CFF0006BDAC3F3130040F4801B0098924620B113
:10D000000023D2EB030A63EB0B0B01985946C0F1E6
:10D010004002504600F0B2F806460D4650465946CA
:10D02000019A00F0BAF810EB08006141002487EA89
:10D03000115284EAE7731A4340D0009A62B3019A0E
:10D04000012A4FEA075215DC001B61EB02014FF089
:10D05000004202EA0752CDE90042001C41F580116E
:10D0600032462B46FFF753FF03B0BDE8F08F404632
:10D070002146F9E7001B61EB0201001C41F580131A
:10D0800000185B412018A2F5001747EB030140EAA6
:10D09000D570B6196D4111E06D084FEA360645EAC4
:10D0A000C0754FEA0752001B61EB0201001C41F5FD
:10D0B000801149084FEA30000019514132462B4691
:10D0C00003B0BDE8F04FFFF713BF00980122400006
:10D0D0000023D0EB020263EBE073009821464FEA95
:10D0E000E074B8EB000061EB0401E9E783F0004372
:10D0F0005BE781F0004158E7C1F30A52C1F3130125
:10D1000040F2FF3341F480119A4202DA00200146D6
:10D11000704740F233439A42A2F2334202DC524259
:10D12000FFF79FBE00F02AB830B5041E71F100046D
:10D1300004DB4FF00044404264EB0101141E73F124
:10D14000000405DB1C464FF00043524263EB04032E
:10D15000994208BF904230BD064C074D06E0E0689A
:10D1600040F0010394E8070098471034AC42F6D32E
:10D17000FFF7E2FB7C3901089C390108202A04DB17
:10D18000203A00FA02F1002070479140C2F12003DA
:10D1900020FA03F3194390407047202A06DBCB178F
:10D1A000203A41FA02F043EAE07306E041FA02F362
:10D1B000D040C2F12002914008431946704770B533
:10D1C0008C1810F8015B15F0070301D110F8013B32
:10D1D0002A1106D110F8012B03E010F8016B01F8B9
:10D1E000016B5B1EF9D12B0705D40023521E0DD411
:10D1F00001F8013BFAE710F8013BCB1A921C03E05F
:10D2000013F8015B01F8015B521EF9D5A142D8D396
:10D21000002070BD21B1826842F00102826003E00B
:10D22000826822F0010282607047014600208A680D
:10D2300002F004020AB1012000E00020704701461C
:10D24000C86C80B270470246002013680B400BB1D7
:10D25000012000E000207047014600208A6802F0AB
:10D2600008020AB1012000E00020704730B50246F4
:10D270000020002350680F4C20400D790C6844EAD0
:10D2800005242043506090680B4C2040D1E90254A3
:10D290002C434D7944EA450420439060D06A20F441
:10D2A00070000C7C641EE4B2234340EA0350D06259
:10D2B00030BD0000FFFEF0FFFDF7F1FFF0B50446C2
:10D2C0000D4600200021092D11DDE068A5F10A06B8
:10D2D00006EB4607072606FA07F18843A5F10A067A
:10D2E00006EB460603FA06F10843E0600CE020690D
:10D2F00005EB4507072606FA07F1884305EB4506C7
:10D3000003FA06F108432061072A0FDA606B561E04
:10D3100006EB86071F2606FA07F18843561E06EB22
:10D32000860605FA06F10843606322E00D2A0FDA4B
:10D33000206BD61F06EB86071F2606FA07F18843E7
:10D34000D61F06EB860605FA06F10843206310E0B7
:10D35000E06AA2F10D0606EB86071F2606FA07F122
:10D360008843A2F10D0606EB860605FA06F108438E
:10D37000E062F0BD816841F008018160704721B131
:10D38000826842F4A002826003E0826822F4A00274
:10D3900082607047816841F004018160704700003D
:10D3A00030B10749096841F40001054A116005E000
:10D3B0000349096821F40001014A11607047000027
:10D3C0000824014010B501221021024800F094FA0F
:10D3D00010BD00000008014010B5002210210248D5
:10D3E00000F08AFA10BD00000008014000BFFEE70F
:10D3F0007047000010B5012000F072F868B10120FC
:10D4000000F068F80548046804E000210846226836
:10D4100090476468002CF8D100BF10BDB400002014
:10D4200010B5022000F05CF868B1022000F052F85C
:10D430000548046804E000210846226890476468B3
:10D44000002CF8D100BF10BDF400002010B504205E
:10D4500000F046F868B1042000F03CF80548046884
:10D4600004E000210846226890476468002CF8D147
:10D4700000BF10BDFC00002010B5202000F030F8E7
:10D4800068B1202000F026F80548046804E0002177
:10D490000846226890476468002CF8D100BF10BD90
:10D4A000040100200949096829B908490860096888
:10D4B000074A116008E005490968814204D0034920
:10D4C000096848600149086070470000F0000020CA
:10D4D000F400002001490860704700001404014076
:10D4E000014600200022074B1B6803EA0102054B9E
:10D4F00014331B680B4013B10AB1012000E0002077
:10D500007047000000040140002123498279002A6D
:10D510003AD00A46126803689A430B461A600A1DFD
:10D52000126803689A430B1D1A60027911440A6855
:10D5300003681A430A60184A0832126803689A435B
:10D54000154B08331A601A1D126803689A43124B70
:10D550000C331A604279102A0ED11A1F1268036820
:10D560001A430D4B08331A601A1D126803681A43D8
:10D57000094B0C331A600DE00749427911440A68DF
:10D5800003681A430A6005E0027911440A680368D7
:10D590009A430A6070470000000401400121034AD9
:10D5A000D1700A21B0FBF1F1D1607047840F0020E7
:10D5B0000549897831B90121034A91700A21B0FBEC
:10D5C000F1F1D16070470000840F00200120014973
:10D5D00008707047840F002030B5044604254FF4CE
:10D5E000302000F06FF80546042D17D10C48006973
:10D5F00040F002000A49086108464461006940F0B1
:10D60000400008614FF4302000F05CF80546044803
:10D61000006941F6FD71084001490861284630BDA6
:10D620000020024004200B49C96801F0010109B142
:10D6300001200EE00749C96801F0040109B1022088
:10D6400007E00449C96801F0100109B1032000E0B6
:10D6500004207047002002400348006940F0800029
:10D6600001490861704700000020024070B504467F
:10D670000D460426F00200F025F80646042E11D1CE
:10D680000948006940F00100074908612580F0025F
:10D6900000F018F806460448006941F6FE7108409B
:10D6A00001490861304670BD00200240024803492C
:10D6B00048600348486070472301674500200240E6
:10D6C000AB89EFCD00B502460423FFF7ABFF03465D
:10D6D00003E0FFF7A7FF0346521E012B01D1002AEA
:10D6E000F7D102B90523184600BD000030B500226D
:10D6F0008B071C0F0F2303FA04F20B4B8C1053F80B
:10D7000024309343084C8D1044F8253023468C1068
:10D7100053F824308C07240F00FA04F42343024CFE
:10D720008D1044F8253030BD080001402DE9F0414E
:10D73000024600250026002000230024002791F83F
:10D7400003C00CF00F0591F803C00CF0100CBCF1F5
:10D75000000F03D091F802C04CEA050591F800C013
:10D76000BCF1000F31D0146800202BE04FF0010C09
:10D770000CFA00F3B1F800C00CEA03069E4220D177
:10D7800083004FF00F0C0CFA03F7BC4305FA03FCBF
:10D790004CEA040491F803C0BCF1280F06D14FF005
:10D7A000010C0CFA00FCC2F814C00AE091F803C0A6
:10D7B000BCF1480F05D14FF0010C0CFA00FCC2F887
:10D7C00010C0401C0828D1D31460B1F800C0BCF1CF
:10D7D000FF0F34DD546800202EE000F1080C4FF0FC
:10D7E000010808FA0CF3B1F800C00CEA03069E42E7
:10D7F00021D183004FF00F0C0CFA03F7BC4305FA5C
:10D8000003FC4CEA040491F803C0BCF1280F05D1D5
:10D8100000F1080C08FA0CF8C2F8148091F803C063
:10D82000BCF1480F07D100F1080C4FF0010808FACD
:10D830000CF8C2F81080401C0828CED35460BDE814
:10D84000F0810000F0B50A460023002400210025E5
:10D8500000F00046B6F1004F02D11D4EF16901E023
:10D860001B4E7168C0F3034583B200F44016B6F551
:10D87000401F08D121F07061154E766826F0706661
:10D88000134F7E6012E000F48016B6F5801F06D1BB
:10D89000032606FA05F4A14341F0706106E0460D47
:10D8A000360103FA06F6B14341F0706122B1460D2C
:10D8B000360103FA06F6314300F00046B6F1004F98
:10D8C00002D1034EF16101E0014E7160F0BD000034
:10D8D000000001400246002093680B400BB101207C
:10D8E00000E00020704702460020D3680B400BB1D7
:10D8F000012000E0002070470AB1016100E04161B1
:10D90000704700BFFEE700000146394841750069D5
:10D9100028B137480069401E354A106102E00020F6
:10D92000334A50703248407D002842D03048C068A9
:10D9300020B12F48C068401E2D4AD0602C48407D41
:10D940002B4A127D90421AD12948807858B1284834
:10D95000C06840B92648807910B90120254A107066
:10D960000120234A90712248C07898B12048C068AD
:10D9700080B901201F4A10701D4AD0710AE01C486E
:10D98000407838B11A48006920B10120194A107056
:10D99000174A50711648007A10B90120154A1070C4
:10D9A0001348407D124A107500201071012010723A
:10D9B00017E00F48007840B10D48007A48B10120C7
:10D9C0000C4A10700A4A107103E00948407D084A69
:10D9D00010750020064AD07090709071D07150710F
:10D9E00010720348007D034A5070104670470000D3
:10D9F000840F0020A101002010B501220821024857
:10DA0000FFF77AFF10BD00000008014010B50022AA
:10DA100008210248FFF770FF10BD00000008014018
:10DA200010B5FFF7F3FF0B48007820F00100401C11
:10DA3000084908700121074881811921C180808827
:10DA400018B90448C0880349888000210148018131
:10DA5000418110BD7001002010B50122082102484B
:10DA6000FFF74AFF10BD00000010014010B5002272
:10DA700008210248FFF740FF10BD000000100140E0
:10DA800010B5FFF7F3FF0B48007820F00200801C70
:10DA90000849087001210748018419214183008B3E
:10DAA00010B90448418B0183002102488183C1835E
:10DAB00010BD00007001002008B50820ADF800007E
:10DAC00010208DF8030003208DF8020069460D48F0
:10DAD000FFF72CFE0820ADF8000010208DF80300A1
:10DAE00003208DF8020069460748FFF71FFE012258
:10DAF00008210448FFF700FF012208210248FFF730
:10DB0000FBFE08BD000801400010014000BFFEE719
:10DB10007047000070B5002100230F22C47804B3C1
:10DB2000154C246804F4E064C4F5E064210AC1F1F2
:10DB30000403CA40447804FA03F184781440214372
:10DB400009010E4C0678A155047804F01F05012444
:10DB5000AC4005786D11AD0005F1E025C5F8004138
:10DB600009E0047804F01F050124AC40044D067858
:10DB7000761145F8264070BD0CED00E000E400E0B1
:10DB800080E100E002490143024A11607047000051
:10DB90000000FA050CED00E010B5FFF713FC0024BF
:10DBA00000E0641C0A2CFCD3FFF716FC002400E004
:10DBB000641C0A2CFCD3FFF705FC002400E0641C65
:10DBC000C82CFCD3302000F0A5FA002400E0641C2F
:10DBD000B4F5FA6FFBD310BD70470000014600207A
:10DBE000034A506820F440400843506070470000EA
:10DBF0000010024029B1064AD2690243044BDA619F
:10DC000004E0034AD2698243014BDA6170470000A5
:10DC10000010024029B1064A92690243044B9A61FE
:10DC200004E0034A92698243014B9A617047000005
:10DC30000010024030B500210022002400232D4DA9
:10DC40006D6805F00C0121B1042905D0082923D104
:10DC500005E0294D056022E0274D05601FE0254DB8
:10DC60006D6805F47012234D6D6805F4803402254B
:10DC700005EB92421CB9214D554305600BE01D4D4B
:10DC80006D6805F400351DB11C4D5543056002E07B
:10DC9000194D5543056002E0174D056000BF00BFF8
:10DCA000144D6D6805F0F0010909154D6B5C0568B0
:10DCB000DD4045600F4D6D6805F4E061090A104DC7
:10DCC0006B5C4568DD4085600A4D6D6805F4605108
:10DCD000C90A0B4D6B5C4568DD40C560054D6D683C
:10DCE00005F44041890B074D6B5CC568B5FBF3F546
:10DCF000056130BD0010024000127A0000093D00AD
:10DD00005C0100206C0100202DE9F04105460E4623
:10DD10001746FFF761FB002401E0601CC4B2642CCD
:10DD2000FBDB45F0C005284604F02AFA002405E094
:10DD3000FF2004F025FA3055601CC4B2BC42F7DB6A
:10DD4000FFF740FBBDE8F08170B50446FFF744FBE8
:10DD5000002501E0681CC5B2642DFBDB44F08004A3
:10DD6000204604F00DFAFF2004F00AFA0646FFF7F9
:10DD700029FB304670BD70B50446FFF72DFB00252A
:10DD800001E0681CC5B2642DFBDB44F0C0042046F2
:10DD900004F0F6F9FF2004F0F3F90646FFF712FB52
:10DDA000304670BDF8B505460E46362000F0B2F993
:10DDB0003B20FFF7E0FF044604F07F0000B33F2064
:10DDC000FFF7C2FF0446B44215DA2C702246691CE4
:10DDD0003F20FFF799FF022269463F20FFF794FF9B
:10DDE0009DF80000094908703A2000F093F99DF869
:10DDF0000100C009F8BD3A2000F08CF90020F9E7D5
:10DE00003A2000F087F90020F4E70000FD0100202F
:10DE100010B5FFF7C1FE01F08BFD362000F07AF956
:10DE20003A2000F077F93B2000F074F9332000F03D
:10DE300071F9082207493E2000F021FE06490878C2
:10DE4000FFF782FF04494978884201D000BFFEE70E
:10DE500010BD0000F40100205039010821B10288F2
:10DE600042F04002028004E002884FF6BF731A407D
:10DE7000028070470246002013890B400BB101203D
:10DE800000E0002070470146888970478181704713
:10DE900010B50022028802F441520B884C882343BB
:10DEA0008C882343CC8823430C8923434C89234308
:10DEB0008C892343CC8923431A430280838B4FF2FE
:10DEC000FF74234083830B8A038210BD30B5034661
:10DED0000C461546002207E0184600F008F824F822
:10DEE00012009B1C501C82B2AA42F5DB30BD0146D9
:10DEF000088870472DE9F05F80468A461746B8F1DA
:10DF0000006F02D33348804501D3BDE8F09FFFF78F
:10DF1000CDFBA8F1006B4FEADB25CBF34909C9F52E
:10DF20008064A74200DC3C464DE04FF0006101EB0D
:10DF3000C5204A142849FFF7C9FF00260BE009EB6A
:10DF40000600254931F810004FF6FF71884200D0D5
:10DF500003E0701C86B2A642F1DB00BFA6421BDACA
:10DF60004FF0006101EBC520FFF736FB002608E00B
:10DF70003AF8160006EB0901174A22F81100701C46
:10DF800086B2A642F4DB4FF0006101EBC5204A14D3
:10DF9000114900F023F804E022465146404600F0C3
:10DFA0001DF8A74200D10FE06D1C4FF000090AEBED
:10DFB000440AA044381B87B2B7F5806F02DD4FF4E6
:10DFC000806400E03C46B0E700BFFFF745FB00BFC0
:10DFD0009BE7000000000408840700202DE9F041C1
:10DFE00005460E461746002407E036F8141028466A
:10DFF000FFF73CFBAD1C601C84B2BC42F5DBBDE806
:10E00000F081704770B504460D46362000F082F866
:10E010003B2000F07FF82A4621463F2000F02FFDEC
:10E02000352000F077F8012070BD10B500F002F83F
:10E0300010BD00000CB5002001900090334800682E
:10E0400040F480303149086000BF3048006800F477
:10E05000003000900198401C0190009818B9019878
:10E06000B0F5A06FF1D12948006800F4003010B17C
:10E070000120009001E0002000900098012843D189
:10E080002348006840F010002149086008460068F5
:10E0900020F0030008600846006840F002000860B5
:10E0A0001A48406819494860084640684860084670
:10E0B000406840F4806048600846406820F47C1066
:10E0C00048600846406840F4E81048600846006828
:10E0D00040F08070086000BF0C48006800F00070DD
:10E0E0000028F9D00948406820F00300074948603B
:10E0F0000846406840F00200486000BF034840689E
:10E1000000F00C000828F9D10CBD000000100240FE
:10E110000020024070B50546FFF75EF9002401E0DB
:10E12000601CC4B2642CFBDB284604F029F8FFF71E
:10E1300049F970BD7047000010B51348006840F001
:10E1400001001149086008464068104908400E491E
:10E150004860084600680E4908400B4908600846B8
:10E16000006820F4802008600846406820F4FE0023
:10E1700048604FF41F008860FFF757FF4FF00060C2
:10E180000449086010BD0000001002400000FFF8C4
:10E19000FFFFF6FE08ED00E0F0B50C461546002244
:10E1A0000021068C4FF6FE773E400684028B018CE0
:10E1B0004FF60C7632407E1C06EA03162E4332439D
:10E1C000104EB0420ED0104EB0420BD0B0F1804F86
:10E1D00008D00E4EB04205D00D4EB04202D00D4ECA
:10E1E000B04206D14FF6FD76314044F0010631438E
:10E1F00005E04FF6F576314044F0010631430283E5
:10E200000184F0BD002C01400034014000040040B6
:10E2100000080040000C0040F0B50C4615460022F6
:10E2200000210026078C4FF6EF7C07EA0C070784D5
:10E23000028B018C4FF6FF7707EA041640F6FF4782
:10E240003A404FF6FF7707EA03373A434FF6FF7736
:10E2500007EA05273A43114FB8420ED0104FB84293
:10E260000BD0B0F1804F08D00E4FB84205D00E4F02
:10E27000B84202D00D4FB84206D14FF6DF77394091
:10E2800046F01007394305E04FF65F77394044F018
:10E290001007394302830184F0BD0000002C0140C7
:10E2A000003401400004004000080040000C004021
:10E2B000F0B50C461546002200210026078C4FF6CB
:10E2C000FF6C07EA0C070784828B018C4FF6FF77FF
:10E2D00007EA04264FF60C773A404FF6FF7707EA35
:10E2E00003172F433A43114FB8420ED0104FB84294
:10E2F0000BD0B0F1804F08D00E4FB84205D00E4F72
:10E30000B84202D00D4FB84206D14FF6FF57394000
:10E3100046F48077394305E04FF2FF57394044F423
:10E320008077394382830184F0BD0000002C0140D6
:10E33000003401400004004000080040000C004090
:10E34000F0B50C461546002200210026078C4EF63B
:10E35000FF7C07EA0C070784828B018C4FF6FF775E
:10E3600007EA043640F6FF473A404FF6FF7707EAE0
:10E3700005273A434FF6FF7707EA03373A43114F31
:10E38000B8420ED0104FB8420BD0B0F1804F08D039
:10E390000E4FB84205D00E4FB84202D00D4FB842D2
:10E3A00006D14DF6FF77394046F48057394305E0F2
:10E3B00047F6FF57394044F480573943828301843C
:10E3C000F0BD0000002C014000340140000400407A
:10E3D00000080040000C004010B50121094800F081
:10E3E000D4F870B10121074800F0BCF80648046871
:10E3F00004E000210846226890476468002CF8D1A8
:10E4000000BF10BD002C0140BC0000200949096874
:10E4100029B9084908600968074A116008E00549F8
:10E420000968814204D003490968486001490860CD
:10E4300070470000B8000020BC00002010B5082183
:10E44000C80600F0A2F801280ED10821800700F0CC
:10E4500089F81048046804E00021084622689047C3
:10E460006468002CF8D100BF0421080700F08DF883
:10E4700001280ED10421800700F074F806480468D2
:10E4800004E000210846226890476468002CF8D117
:10E4900000BF10BDCC000020C4000020094909685D
:10E4A00029B9084908600968074A116008E0054968
:10E4B0000968814204D0034909684860014908603D
:10E4C00070470000D0000020D400002010B500F0FC
:10E4D000B7FF094801780078401C074A10700529E9
:10E4E00009D100201146087004480068401C034907
:10E4F000086001F071F910BDA8000020280000207C
:10E5000010B51021144800F040F801280ED1102158
:10E51000114800F027F81148046804E0002108467B
:10E52000226890476468002CF8D100BF01210A4896
:10E5300000F02BF870B10121074800F013F80848EB
:10E54000046804E000210846226890476468002CB3
:10E55000F8D100BF10BD000000040040D40000202E
:10E56000DC000020CA430282704721B1028842F0D9
:10E570000102028004E002884FF6FE731A40028016
:10E5800070470146B1F84000704730B502460020A0
:10E5900000230024158A05EA0103958905EA010490
:10E5A00013B10CB1012000E0002030BD70B505466C
:10E5B0000C46244885420ED0234885420BD0B5F145
:10E5C000804F08D02148854205D02148854202D09D
:10E5D0002048854200D100E000BF208850B923893F
:10E5E000A28861882846FFF7D7FDE188284600F019
:10E5F0003CF825E0208804280AD12389A288618874
:10E600002846FFF709FEE188284600F037F817E0B2
:10E61000208808280AD12389A28861882846FFF724
:10E6200047FEE188284600F036F809E02389A288F1
:10E6300061882846FFF784FEE188284600F034F818
:10E6400070BD0000002C0140003401400004004077
:10E6500000080040000C00401AB183890B438381FD
:10E6600002E083898B4383817047028B4FF6F373FB
:10E670001A400283028B0A4302837047028B4FF2D7
:10E68000FF331A400283028B4FF6FF7303EA012324
:10E690001A4302837047828B4FF6F3731A408283CA
:10E6A000828B0A4382837047828B4FF2FF331A407A
:10E6B0008283828B4FF6FF7303EA01231A4382831E
:10E6C00070470000002202881D4B98420ED01D4B5F
:10E6D00098420BD0B0F1804F08D01B4B984205D028
:10E6E0001A4B984202D01A4B984204D14FF68F73BE
:10E6F0001A404B881A43174B984207D0164B984242
:10E7000004D04FF6FF431A40CB881A4302808B880F
:10E7100083850B8803850A4B98420BD0094B98429E
:10E7200008D00E4B984205D00D4B984202D00D4BAD
:10E73000984201D10B7A038601238382704700003F
:10E74000002C01400034014000040040000800405B
:10E75000000C004000100040001400400040014048
:10E76000004401400048014070B505460C46194878
:10E77000007868BB224629461648401CFEF7F4F88C
:10E780001448A0F800410120124908704E1C0846A8
:10E7900090F80011401C00F031FFA8B170785328A8
:10E7A00010D103F003F900BF0B48006800F4E060EB
:10E7B0000A490843001D08490860BFF34F8F00BF96
:10E7C00000BFFEE700BF00BF032001F071F800BFEB
:10E7D00070BD0000240200200CED00E00000FA05EE
:10E7E00070B51348046840F22441124800F081F8E3
:10E7F00058B1104800F038F9054604E029460020D9
:10E80000226890476468002CF8D140F225510948ED
:10E8100000F06FF858B1074800F026F9054604E00B
:10E8200029460120226890476468002CF8D170BD09
:10E83000E4000020003801400949096829B9084965
:10E8400008600968074A116008E0054909688142C3
:10E8500004D0034909684860014908607047000016
:10E86000E0000020E400002070B51348046840F286
:10E870002441124800F03DF858B1104800F0F4F877
:10E88000054604E029460020226890476468002C71
:10E89000F8D140F22551094800F02BF858B107484B
:10E8A00000F0E2F8054604E029460120226890477E
:10E8B0006468002CF8D170BDEC00002000480040D6
:10E8C00021B1828942F40052828104E082894DF6AE
:10E8D000FF731A408281704702460020B1F5007F25
:10E8E00000D100BF13880B400BB1012000E00020D5
:10E8F000704770B50246002400230025002040F632
:10E900006A16B14200D100BFC1F3421501F01F03E6
:10E91000012606FA03F3012D02D19689334006E061
:10E92000022D02D1168A334001E0968A33400C1240
:10E93000012606FA04F41688344013B10CB1012004
:10E9400000E0002070BDF0B503460024002600253D
:10E95000002040F66A17B94200D100BF1846C1F343
:10E96000421401F01F06012707FA06F5012C01D118
:10E970000C3004E0022C01D1103000E014301AB148
:10E9800007682F43076002E00768AF430760F0BDE8
:10E990002DE9F04786B005460E460024A24600BF8A
:10E9A000A1460027B08900B100BF2F462C8A4CF643
:10E9B000FF700440F08804432C82AC894EF6F310BB
:10E9C0000440B08831890843718908430443AC810D
:10E9D000AC8A4FF6FF400440B0890443AC8201A8E2
:10E9E000FFF728F91F48874202D1DDF810A001E0A7
:10E9F000DDF80CA0A88900F4004040B10AEBCA0081
:10EA000000EB0A1031684900B0FBF1F807E00AEBAF
:10EA1000CA0000EB0A1031688900B0FBF1F86420ED
:10EA2000B8FBF0F004012009642101FB1089A889DA
:10EA300000F4004040B1322000EBC900B0FBF1F01F
:10EA400000F00700044308E0322000EB09106421C5
:10EA5000B0FBF1F000F00F0004432C8106B0BDE8DC
:10EA6000F08700000038014001468888C0F30800A4
:10EA70007047C1F308028280704700BFFEE72DE9AE
:10EA8000F04105460E461746FEF7A6FC002401E0BD
:10EA9000601CC4B2642CFBDB25F0800545F040050A
:10EAA000284603F06DFB002404E0305D03F068FBB2
:10EAB000601CC4B2BC42F8DBFEF784FCBDE8F08108
:10EAC00070B504460D46FEF787FC002601E0701C79
:10EAD000C6B2642EFBDB24F08004204603F050FB1A
:10EAE000284603F04DFBFEF76DFC70BD7CB5044677
:10EAF00000201D46164600290BD0491ECDE90041D5
:10EB0000044B6A462946304600F0DAF8009A0021A4
:10EB100011707CBDEFF3000802E008C8121F08C1A5
:10EB2000002AFAD170477047002001E001C1121F8E
:10EB3000002AFBD1704780F3108870472DE9FF5FF2
:10EB400082B00021DDE90430020DDDF840B003435E
:10EB500018D044F61050A2F2FF3242431514119817
:10EB600001281FD0A5EB0B00401C5FEA000A4FF004
:10EB700000064E4FDFF83891B046504615D5CAF121
:10EB8000000413E0119801244AA3012801D16FEA7F
:10EB90000B010298119AC0E90031C0E9024206B0A7
:10EBA000BDE8F09FCBF10000DFE704460021404ABA
:10EBB000491842EB0450CDE9001012E0E00707D0FD
:10EBC00032463B4640464946FDF7CEFF80468946E1
:10EBD00032463B4610461946FDF7C6FF06460F462D
:10EBE0006410002CEAD1DDE90401DDE90023BAF16B
:10EBF000000F06DAFDF7B8FF42464B46FDF7B4FFBB
:10EC000005E0FEF723F842464B46FEF71FF80446A0
:10EC10000E460022284BFEF787FA03D84FF0FF304C
:10EC2000014607E00022254B20463146FEF7BDF99C
:10EC3000FEF762FA102409E0002C0ADB0A22002306
:10EC4000FEF7DEF8039B30321A55641E50EA0102CB
:10EC5000F2D1641C039AC4F111031444119A012ADD
:10EC600003D0012208430DD10AE0084304D000205C
:10EC70004FF0110B119072E7A3EB0B056D1E0DE029
:10EC80005B4504DD4FF0000205F1010504E003DA05
:10EC90004FF00002A5F10105002AECD0029811996D
:10ECA000C0E90231C0E9004579E7000000001440E6
:10ECB0000000F03F300000000000F0430000E03FA3
:10ECC0002DE9FF4F95B09B468946064600250FE289
:10ECD000252877D100242746F84A0121059400E031
:10ECE000044316F8013F203B01FA03F01042F7D12C
:10ECF00030782A2811D06FF02F033078A0F130023D
:10ED0000092A16D8059A44F0020402EB820203EBAA
:10ED100042021044761C0590EFE759F8042B059247
:10ED2000002A03DA504244F40054059044F00204EF
:10ED3000761C30782E2816D116F8010F44F0040402
:10ED40002A280DD06FF02F023078A0F13003092B64
:10ED500009D807EB870302EB4303C718761CF3E7D8
:10ED600059F8047B761C30786C280FD006DC4C28D0
:10ED700017D068280DD06A2814D104E0742810D068
:10ED80007A280FD10DE044F400140AE044F4801412
:10ED900001E044F440147278824202D104F58014F8
:10EDA000761C761C307866280BD013DC582877D078
:10EDB00009DC002875D04528F6D04628F4D047282D
:10EDC0001AD19DE118E0632835D0642879D06528F0
:10EDD00012D195E1702873D008DC6728F1D069283A
:10EDE0006FD06E280DD06F2806D1B5E073282CD0D7
:10EDF000752875D0782874D05A46179990476D1C9D
:10EE000075E1C4F30250022809D003280DD0D9F8C7
:10EE1000001004280DD00D6009F1040967E1D9F84C
:10EE20000010EA17C1E90052F6E7D9F800100D808A
:10EE3000F2E70D70F0E719F8041B8DF800100020C0
:10EE40008DF80100EA46012003E059F804AB4FF0C9
:10EE5000FF3061074FF0000102D40DE008F101011D
:10EE60008846B9420FDA8045F8DB1AF80810002905
:10EE7000F4D108E008F1010188468142FADB1AF872
:10EE800008100029F6D105985B46A0EB080721463B
:10EE90003846179A00F094FA284400EB080507E07A
:10EEA0004DE029E10DE01AF8010B5A4617999047F9
:10EEB000B8F10108F7D25B4621463846179A13E1AC
:10EEC00042E00A220092C4F302524FF0000A022AE2
:10EED00008D059F804CB032A4FEAEC710AD00DE0B0
:10EEE00029E02AE009F1070121F00702F2E802C156
:10EEF000914609E00FFA8CFC4FEAEC71042A03D129
:10EF00004FFA8CFC4FEAEC71002907DA0A4600211F
:10EF1000DCF1000C61EB02012D2202E0220504D598
:10EF20002B228DF80420012203E0E20701D02022E9
:10EF3000F7E7904659E00A2102E010220DE0102187
:10EF40004FF0000A00910BE010224FF0000A44F04D
:10EF500004040827009203E008224FF0000A009200
:10EF6000C4F30252022A05D059F804CB0021032A27
:10EF700008D009E009F1070121F00702F2E802C117
:10EF8000914605E01FFA8CFC042A01D10CF0FF0C1D
:10EF90004FF00008220728D5702806D0009B83F088
:10EFA000100353EA0A0305D00EE040228DF8042036
:10EFB000012208E05CEA010206D030228DF804202C
:10EFC0008DF8050002229046009B83F0080353EA67
:10EFD0000A030AD15CEA010201D1620705D5302299
:10EFE0008DF804204FF001087F1E582804D034A06B
:10EFF00003900EA802900DE036A0F9E75346604654
:10F00000009AFDF7FDFE84460398825C0298401E3C
:10F01000029002705CEA0100F0D1029806A9081A79
:10F0200000F1200A600702D524F4803400E00127B3
:10F03000574502DDA7EB0A0000E0002000EB0A01C3
:10F04000009005984144401A0590E00306D45B46C1
:10F050002146179A059800F0B3F90544002706E009
:10F0600001A85A46C05D179990476D1C7F1C474503
:10F07000F6DBE0030CD55B462146179A059800F0B5
:10F080009FF9054404E030205A46179990476D1CBB
:10F090000099481E00900029F5DC08E002980299CA
:10F0A0005A460078491C0291179990476D1CBAF195
:10F0B0000001AAF1010AF1DC65E100000928010064
:10F0C00030313233343536373839616263646566DE
:10F0D00000000000303132333435363738394142A0
:10F0E000434445460000000000F058F90544761CF2
:10F0F000307800287FF4ECAD19B02846BDE8F08FD9
:10F10000620700D4062709F1070222F0070CFCE889
:10F110000223E14603F000485FEA080C02D00FF238
:10F12000702C0DE05FEA045C02D50FF2682C07E05A
:10F130005FEAC47C02D00FF2602C01E0AFF2700CE9
:10F140004FF0FF3823F00043CDF850C065280CD0B5
:10F1500006DC452809D046281DD047283DD13DE092
:10F16000662818D067287ED138E00021112F01DBF6
:10F17000112000E0781CCDE9000106A90EA8FFF7D8
:10F18000DDFCDDE90F010E9A03910021009207F1E9
:10F19000010A04914DE04FF000400097CDE90110C5
:10F1A00006A90EA8FFF7CAFCDDE90F0203920E9B29
:10F1B00011990022DDF80CA00093049211B9791C7A
:10F1C00000EB010AB7EB0A0004D4C0F1FF3007F1ED
:10F1D000010A0490AAEB0700019044E0012F00DA35
:10F1E00001270021112F01DD112000E03846CDE973
:10F1F000000106A90EA8FFF7A1FCDDE90F010E9A98
:10F200000391002104910092BA4621070CD403997E
:10F21000514500DA8A46BAF1010F05DD009AAAF1DC
:10F220000101515C302908D0B84202DA10F1040F14
:10F2300006DA0121CDE9011015E0AAF10101E9E7A3
:10F24000002805DC049901440491AAEB000102E0C6
:10F25000411C514500DD8A460499401A401C01902A
:10F260004FF000400290200704D40198504501DB84
:10F27000CDF8048000208DF84F0002980DF14F0763
:10F28000B0F1004F25D02B200E9002984FF00208CD
:10F2900000280CDA404202902D200E9007E00A214F
:10F2A0000298FDF797FD3031029007F8011DB8F183
:10F2B0000001A8F10108F2DC02980028EFD1791EC4
:10F2C0000E980870307800F0200040F0450007F8F4
:10F2D000020D12A8C01B00F107081498007800B1B5
:10F2E000012000EB0A01019801EBE071059841440F
:10F2F000401A401E0590E00306D45B462146179A4B
:10F30000059800F05DF805441498007818B15A4645
:10F31000179990476D1CE00324D55B462146179A48
:10F32000059800F04DF805441CE00498002807DB20
:10F33000DDE90301884203DD0098405C179901E094
:10F34000179930205A469047049805F10105401C52
:10F3500004900198401E019004D12E205A4617991E
:10F3600090476D1CBAF10001AAF1010ADDDC05E04D
:10F3700017F8010B5A46179990476D1CB8F1000118
:10F38000A8F10108F4DC5B462146179A0598ABE624
:10F390002D0000002B000000200000002DE9F041AE
:10F3A000044600251E461746880404D405E0394665
:10F3B0002020B0476D1C641EF9D52846BDE8F081B9
:10F3C0002DE9F041044600251E469046C80301D5AC
:10F3D000302700E02027880404D505E04146384660
:10F3E000B0476D1C641EF9D52846BDE8F0814A6817
:10F3F000002A06D00A68531C0B6010704868401E33
:10F400004860704708B54FF48050ADF800001020F8
:10F410008DF8030003208DF8020069460448FEF7CA
:10F4200085F900224FF480510148FEF765FA08BDC6
:10F4300000080140C8200149088070479C01002055
:10F4400010B563480078401C614908700846007890
:10F4500060490978884215DB00205D4908705E48E4
:10F46000008878B14FF480515C48FEF73CFA08B947
:10F47000012000E00020044622464FF48051574806
:10F48000FEF73AFA5448008868B153480088401E95
:10F49000514908800846008828B900224FF480515D
:10F4A0004E48FEF729FA00248EE004EB84014C4814
:10F4B00030F82100002858D004EB8401484830F887
:10F4C0002100401E81B204EB8402454820F822103E
:10F4D00004EB840130F82100002874D104EB84018E
:10F4E0003F4800EB8100008900286CD004EB8402C7
:10F4F0003B4901EB82010869804704EB84013848ED
:10F5000000EB81000089401E81B204EB8402344884
:10F5100000EB8200018104EB8401314800EB8100A3
:10F520000089A8B92E48001F00780121A140884316
:10F530002B49091F097860F300012948001F017059
:10F54000002104EB8402001D00EB820081803AE080
:10F5500004EB8401224800EB8100C18804EB8402A3
:10F560001F4800EB820081802DE004EB84011C48E1
:10F5700000EB8100808830B304EB8401184800EB75
:10F5800081008088401E81B204EB8402144800EBA5
:10F590008200818004EB8401114800EB81008088A7
:10F5A00088B904EB84010E4800EB8100418804EB2C
:10F5B00084020B4820F8221004EB8402014601EB80
:10F5C000820108698047641C022CFFF66EAF10BDF3
:10F5D0009F0100209E0100209C01002000080140A6
:10F5E0007401002001490870704700009E0100204E
:10F5F0003C200149088070479C0100202DE9F04320
:10F6000004460D460027267894F8018014F80690E9
:10F61000681EB0420CD108F0800040B9681E81B26B
:10F620004A46204600F00EF810B1012700E00127FD
:10F630003846BDE8F083000000200149887070471B
:10F64000840F002070B505460E4614460723552248
:10F650003146284600F006F8A04201D1012070BDD5
:10F660000020FCE7F0B50446104611E014F8016BE9
:10F67000704000250AE000F080061EB14606300EFC
:10F68000584001E04606300E6E1CF5B2082DF2DB44
:10F690000E1EA1F10101E9D1F0BD30B504460D46C1
:10F6A0003123FF2229462046FFF7DCFF30BD70B52D
:10F6B00005460E4614463123FF2231462846FFF701
:10F6C000D1FFA04201D1012070BD0020FCE7000065
:10F6D00010B540480068007800B910BD00203D49D1
:10F6E000096808703B480068407806286DD2DFE85A
:10F6F00000F06C24033E155800F00EF938B1FFF706
:10F700009BFFFDF763FF012001F076F805E000F0B4
:10F7100009F910B90520FDF74BFF57E000F0FCF8A0
:10F7200020B1FFF789FFFDF751FF05E000F0FAF87F
:10F7300010B90520FDF73CFF48E000F0DDF830B1DE
:10F740001E20FDF72BFF012000F0E8FD0EE000F089
:10F75000E9F828B1FFF74CFF012000F0DFFD05E0DC
:10F76000FDF734FF4FF49670FDF718FF2EE000F020
:10F77000C3F830B11E20FDF711FF002000F0CEFDD0
:10F780000EE000F0CFF828B1FFF732FF002000F0C4
:10F79000C5FD05E0FDF71AFF4FF49670FDF7FEFE7C
:10F7A00014E000F0B9F848B1FFF746FFFDF70EFF8F
:10F7B000FFF71EFF002001F01FF805E000F0B2F88F
:10F7C00010B90520FDF7F4FE00E000BF00BF00BF48
:10F7D00083E7000000000020002034E000EB40013F
:10F7E0001A4A02EB8101896861B300EB400102EB28
:10F7F00081014968491C00EB4002144B03EB820273
:10F80000516000EB400203EB82029268521E91426B
:10F8100018D3002100EB400203EB8202516000EBA1
:10F8200040011A4612F8211029B9002100EB4002CC
:10F8300003EB8202916001218140054A1268114365
:10F84000034A1160401C2028C8DB7047C40F002009
:10F85000BC01002010B504460120FFF76CF9002020
:10F8600004EB4401074A02EB8101886004EB440188
:10F8700002EB8101486004EB440102F82100FFF72C
:10F880005AF910BDC40F002010B500240120FFF765
:10F8900052F90548046805480460002002490860E0
:10F8A000FFF749F9204610BDBC010020C00100202F
:10F8B00010B504460120FFF73EF9002004EB440197
:10F8C0000B4A02EB8101886004EB440102EB8101E9
:10F8D000486004EB440102F821000120A0400549E2
:10F8E00009680843034908600020FFF724F910BDA8
:10F8F000C40F0020BC0100200148C07970470000FF
:10F90000840F0020014601208840024A12681040FE
:10F9100070470000C0010020014880797047000056
:10F92000840F00200148007970470000840F0020F8
:10F9300010B500240AE0074A02EB44025178054A58
:10F9400012F81400FFF7BCF8601C84B2162CF2D336
:10F9500010BD00005039010810B5002401211248E3
:10F96000FDF7B8FF08B901241CE04FF480410F48AF
:10F97000FDF7B0FF08B9022414E04FF400410B4832
:10F98000FDF7A8FF08B903240CE040210848FDF763
:10F99000A1FF08B9042405E080210548FDF79AFF7E
:10F9A00000B90524204610BD00080140000C0140AC
:10F9B0000010014008B50120ADF8000048208DF886
:10F9C000030069461648FDF7B1FE4FF48040ADF8DC
:10F9D000000048208DF8030069461248FDF7A6FE96
:10F9E0004FF40040ADF8000048208DF80300694650
:10F9F0000C48FDF79BFE4020ADF8000048208DF834
:10FA0000030069460848FDF791FE8020ADF800002C
:10FA100048208DF8030069460348FDF787FE08BDBE
:10FA200000080140000C01400010014070B5044680
:10FA30000D4614220B49A1F11400FCF795FF142286
:10FA4000084914310748FCF78FFF1421054814308A
:10FA5000FCF7A3FF1422214602481430FCF784FF70
:10FA600070BD00009C15002070B504460D461422A0
:10FA70000749A1F11400FCF777FF14210448FCF7B3
:10FA80008CFF142221460248FCF76EFF70BD000077
:10FA90009C150020FC48FD4908604FF4A060FEF76B
:10FAA00071F802F011FE0121F948FDF7CBFE1F218C
:10FAB000F84801F059FFF748827F1E21FFF7F7FD54
:10FAC00020B91F22F449F348FCF74EFFF248FCF737
:10FAD0006FFF04462246F049EE48FCF770FF20B164
:10FAE0001F22ED49EB48FCF73FFFFFF763FFFDF7EF
:10FAF000E3FFEA494FF4E13002F064FDE849C82031
:10FB000002F022FD00F0BCFBFFF77CFCE149487FDE
:10FB1000FFF768FDDF49087F02F09EFCE149002005
:10FB200002F010FCDB49087E02F0DCFCD94991F9B7
:10FB30001A10DD4A505602F0E7FCD649C87E02F0A2
:10FB40007FFCDA4801F038F8D249097F01EB8101E6
:10FB5000D74A02EB810001F0F9F9CE49097ECD4A7E
:10FB6000527E11FB02F101EB8101490001EB4102E0
:10FB7000C2EBC111C74A127FCE4B53F8222002EBD1
:10FB8000C10001F0EDF9C34991F91A10C64A505667
:10FB900001F028FABF49C97EC74A52F8210001F096
:10FBA00001FABC48017F04230022104601F00AF943
:10FBB000B848017E1F230022012001F003F9B54857
:10FBC000417E15231422022001F0FCF8B14890F97F
:10FBD0001A1009230022032001F0F4F8AD48C17E79
:10FBE00007230222042001F0EDF8AA49097EA94A60
:10FBF000527E11FB02F101EB8101490001EB410250
:10FC0000C2EBC111A34A127FAA4B53F8222002EB88
:10FC1000C10001F055FD9F49497E01EB810149007A
:10FC20004FF47A7211FB02F001F044FD9949097F0B
:10FC300001EB81019E4A02EB810001F053FD9549E1
:10FC4000C97E9D4A52F8210001F040FD914991F989
:10FC50001A10954A505601F03FFD012001F0C6F8F8
:10FC600096A001F0BDF8FFF7E5FB0A220121002074
:10FC700002F09AFD4FF4FA720121084602F094FD59
:10FC800002F0C6FB93E2FFF7FFFD914908800020D8
:10FC9000FFF738FE38B18F480078FDF735FE8E4902
:10FCA0000860FFF715FD0120FFF72CFE60B300F0A0
:10FCB000BDFA83468949FCF719FF8246FDF75BF8D8
:10FCC00006460022864BFCF7C1FF04460022854B06
:10FCD000FCF74AFF8046FDF761F883490860084653
:10FCE000006801F077FA8048006801F035FB02F007
:10FCF00061FF7E48006801F035FA00207C49086009
:10FD00004FF07E507B4908600620FFF7FBFDF8B1FD
:10FD1000794801F0B1FE5F48007E5E4A527E10FBDA
:10FD200002F000EB8000400000EB4002C2EBC0108C
:10FD3000584A127F5F4B53F8222002EBC00101208A
:10FD400002F090FB01206D490870002068490860AE
:10FD50000520FFF7D7FDB0B14E48007E4D4A527ED8
:10FD600010FB02F000EB8000400000EB4002C2EB11
:10FD7000C010484A127F4F4B53F8222002EBC001BB
:10FD8000002002F06FFB0820FFF7BCFDD8B141490D
:10FD900091F91A0002F0B8FB3E48007E3D4A527EBF
:10FDA00010FB02F000EB8000400000EB4002C2EBD1
:10FDB000C010384A127F3F4B53F8222002EBC0019B
:10FDC000022002F04FFB0B20FFF79CFD00285AD0C9
:10FDD0000B204B4908730846027B4AA10D30FCF703
:10FDE000C3FD4B48007800F00F00303044490A7BD7
:10FDF0000D3188544248007B401C0D3908730021A6
:10FE00003F48027B0D30815401F0D4FC404800682B
:10FE1000FCF78BFF80463F480068FCF786FF814671
:10FE20004146FCF763FE07463B49FCF72DFE0646BC
:10FE30003A49FCF729FE0546FCF789FF0446344899
:10FE40000168204601F0EAFC2D4802F069FB0D2014
:10FE5000FFF700FD32480078022814D12C480068D2
:10FE6000401C2B4908602F48006828B12D480068C5
:10FE700040F2DC51884257D940F2DC5200210B207D
:10FE800002F092FC5DE076E000C8000808ED00E0BA
:10FE900000023000500600208600002069E70008BC
:10FEA000CDE4000821270108482D01081D2901087B
:10FEB000360000201C2D01082C2D010856474B69E7
:10FEC00074426F6172645F3232313253000000005D
:10FED000A60000200400002000000020000048428E
:10FEE0000000E03F00408F400C0000201C0000207C
:10FEF0001400002010000020F5190108080000205F
:10FF00004005002068656C6C6F20776F726C640030
:10FF100020000020240000200000C84200002041F2
:10FF2000350000202C000020A148006800EB800074
:10FF300080000A21B0FBF1F4224600210B2002F0E0
:10FF400033FC00209B4908609B48007880B94FF043
:10FF5000FF3001F03FFC99480068401C9749086059
:10FF6000084600680A2803D100200860904908600C
:10FF70000020914908700C20FFF7C4FC20B102F06A
:10FF800047FA00208E4908600A20FFF7BBFC0028D2
:10FF90007ED08C480068401C8A4908608A49B1F9C3
:10FFA000080001F0B9F98748006801F09FF90021C5
:10FFB0008548153001F0EAF900218348153001F039
:10FFC00023F97F480068FCF7C2FE84B22146002076
:10FFD00001F0E4F87C48017D153002F057FB4FF446
:10FFE000807179481530FCF7D8FC784800780228F1
:10FFF00052D17048006801F0EDFB7349B1F9080077
:020000040801F1
:1000000001F0B8FB72480068FCF78FFE80466D482F
:100010000068FCF78AFE81464146FCF767FD07460B
:100020006C49FCF731FD06466B49FCF72DFD054692
:10003000FCF78DFE044666480168204601F0EEFBA1
:100040005C48006828B15B48006840F2DC51884297
:1000500006D340F2DC5200210B2002F0A5FB0CE09D
:100060005448006800EB800080000A21B0FBF1F4E6
:10007000224600210B2002F097FB01204E49087018
:1000800000204E4908604B4800684949086000E07C
:100090000DE00020474908604C480078032804D14F
:1000A000002211460B2002F07FFBFDF7E9FC0E2039
:1000B000FFF728FC08B102F0ABF90720FFF722FC9C
:1000C00038B100204549087002F084F80B20FFF792
:1000D000C1FB0320FFF716FCF0B341480078D8B30A
:1000E00000203F4908703A480068401C38490860C1
:1000F0003B4890F800013B4908730846007BB0F587
:10010000807F01DD002008733648027B3449491C9A
:100110000D30FCF729FC33480D3001F04BFB2C4827
:100120000068FCF702FE804626480068FCF7FDFDEB
:1001300081464146FCF7DAFC07462649FCF7A4FC59
:1001400006462549FCF7A0FC0546FCF700FE0446E0
:100150001F480168204600E004E001F05FFB2148F1
:1001600002F0DEF90220FFF7CDFB60B11E480078F7
:1001700048B100201C490870A1F8000100211A486C
:10018000401C01F067F80920FFF7BCFB48B11E21B5
:100190001648FFF782FA154988771F21134801F0A6
:1001A00013FCFFF7D9FB1249087002F0E3F86AE587
:1001B0002C00002028000020340000203000002007
:1001C0001400002024000020280400203500002016
:1001D000200000200000C84200002041080000204C
:1001E00024020020400500202603002050060020A5
:1001F0000400002070B504460723012221460A4866
:10020000FDF75CF801210848FDF7B9F800BF0221AD
:100210000548FDF718F80028F9D00348FDF70FF856
:100220000546284670BD0000002401402DE9FF5F0F
:100230001120FFF7DFFF02900120FFF7DBFF0390A3
:100240000298FCF777FD04460D460398FCF76DFD18
:100250000090FCF790FD80464FF03332074BFCF7DF
:1002600083FC064622462B46FCF7F0FC8246FCF750
:1002700095FD0190019804B0BDE8F09F3333F33F42
:1002800008B501214802FDF7C5FC0220ADF80000C9
:1002900000208DF8030069461D48FDF747FA00204D
:1002A0001C490860087148714FF460208860002084
:1002B000C860012008741848FCF7D8FF0523012204
:1002C00011461548FCF7FAFF0523022211211248B6
:1002D000FCF7F4FF01211048FCF79CFF0120FDF71B
:1002E0005FF80D48FDF746F800BF0B48FCF7B4FF78
:1002F0000028FAD10848FDF74DF800BF0648FCF782
:1003000094FF0028FAD101210348FDF738F808BD11
:1003100000080140700700200024014070B5044629
:10032000FB4890F90000401EC0EBC00101EB4010FB
:10033000F84951F8200000287ED0F54890F90000D7
:10034000401EC0EBC00101EB4010F24901EB800000
:100350008E30EF4991F90010491EC1EBC10202EB4A
:100360004111EC4A02EB81014968405C00287CD0D5
:10037000002C7BD0E64890F90000401EC0EBC00185
:1003800001EB4010114601EB80004030E04991F94B
:100390000010491EC1EBC10202EB4111DD4A02EB24
:1003A0008101496850F82110491CD94890F9000092
:1003B000401EC0EBC00202EB4010D64A02EB8000A8
:1003C0004030D34A92F90020521EC2EBC20303EB25
:1003D0004212D04B03EB8202526840F82210CC4804
:1003E00090F90000401EC0EBC00101EB401019461F
:1003F00001EB80004030C64991F90010491EC1EB65
:10040000C10202EB41111A4602EB8101496850F822
:100410002120BF4890F90000401EC0EBC00101EB55
:100420004010194601EB80007030B94991F9001075
:10043000491EC1EBC10300E0D9E103EB4111B54B0B
:1004400003EB8101496850F82100824236DBB04855
:1004500090F90000401EC0EBC00101EB40101946AE
:1004600001EB80005830AA4901E012E127E091F940
:100470000010491EC1EBC10202EB41111A4602EB0A
:100480008101496850F82120A14890F90000401EE0
:10049000C0EBC00101EB4010194601EB8000403079
:1004A0009B4991F90010491EC1EBC10303EB4111B7
:1004B000984B03EB8101496840F821209FE0944864
:1004C00090F90000401EC0EBC00101EB40109149C3
:1004D00001EB800040308E4991F90010491EC1EBBC
:1004E000C10202EB41118B4A02EB8101496850F8CD
:1004F0002110491E864890F90000401EC0EBC00242
:1005000002EB4010834A02EB80004030804A92F9AF
:100510000020521EC2EBC20303EB42127D4B03EBE1
:100520008202526840F82210794890F90000401E7B
:10053000C0EBC00101EB4010194601EB80004030D8
:10054000734991F90010491EC1EBC10202EB411140
:100550001A4602EB8101496850F821206C4890F955
:100560000000401EC0EBC00101EB4010194601EB3A
:1005700080005830664991F90010491EC1EBC10353
:1005800003EB4111634B03EB8101496850F82100F3
:10059000824234DA5E4890F90000401EC0EBC00190
:1005A00001EB4010194601EB80007030584991F979
:1005B0000010491EC1EBC10202EB41111A4602EBC9
:1005C0008101496850F82110491E514890F90000F6
:1005D000401EC0EBC00202EB40101A4602EB800046
:1005E00040304B4A92F90020521EC2EBC20303EB8B
:1005F0004212484B03EB8202526840F822104648F0
:100600000068002844D0424890F90000401EC0EB2A
:10061000C00505EB40103F4D05EB800040303C4DE0
:1006200095F900506D1EC5EBC50606EB4515394E14
:1006300006EB85056D6850F82530354890F90000C7
:10064000401EC0EBC00505EB4010354605EB8000B1
:100650008E302F4D95F900506D1EC5EBC50606EB8B
:1006600045152C4E06EB85056D68425D284890F9CE
:100670000000401EC0EBC00505EB4010354605EB01
:1006800080004168224890F90000234D2D68A8475A
:1006900087E0E4B31E4890F90000401EC0EBC001A3
:1006A00001EB40101B4901EB80004068401E1849D7
:1006B00091F90010491EC1EBC10202EB4111154A2C
:1006C00002EB81014860124890F90000401EC0EB27
:1006D000C00101EB4010114601EB8000406800288A
:1006E0005FDA0B4890F90000401EC0EBC00101EB3F
:1006F0004010114651F82000401E054991F90010A4
:10070000491EC1EBC10202EB4111024A06E009E0B9
:10071000C901002044110020D001002002EB81011A
:1007200048603EE0324890F90000401EC0EBC00136
:1007300001EB40102F4901EB80004068401C2C4920
:1007400091F90010491EC1EBC10202EB4111294A87
:1007500002EB81014860264890F90000401EC0EB82
:10076000C00101EB4010114601EB800041682048B8
:1007700090F90000401EC0EBC00202EB40101D4A81
:1007800052F8200081420CDB0021194890F900004A
:10079000401EC0EBC00202EB4010164A02EB800084
:1007A0004160134B93F900305B1EC3EBC30505EBAF
:1007B0004313104D05EB830303F140010C4B93F9F8
:1007C00000305B1EC3EBC30505EB4313094D05EB7E
:1007D00083035868064B93F900305B1EC3EBC305D7
:1007E00005EB4313034D05EB83039A68904770BDF7
:1007F000C9010020441100202DE9F0410446002CDD
:100800007ED1EA4890F90000401EC0EBC00101EB28
:100810004010E74901EB80008830E44991F900106D
:10082000491EC1EBC10202EB4111E14A02EB810119
:100830004968405C01287CD1DC4890F90000401EEA
:10084000C0EBC00101EB4010114601EB80008E307F
:10085000D64991F90010491EC1EBC10202EB4111CA
:10086000D34A02EB81014968405C08B9012200E0EB
:100870000022CE4890F90000401EC0EBC00101EB01
:100880004010CB4901EB80018E31C84890F900003F
:10089000401EC0EBC00303EB4010C54B03EB8000D0
:1008A00040680A54C14B93F900305B1EC3EBC3058B
:1008B00005EB4313BE4D05EB830303F14001BB4B36
:1008C00093F900305B1EC3EBC30505EB4313B84D32
:1008D00005EB83035868B54B93F900305B1EC3EBFF
:1008E000C30505EB4313B24D05EB83039A689047AC
:1008F000B0480068E8B1AD4D95F900506D1E00E0BC
:10090000A9E0C5EBC50606EB4515A94E06EB850526
:100910004035A64E96F90060761EC6EBC60707EB7B
:100920004616A34F07EB8606766855F826309F4D8E
:1009300000E032E095F900506D1EC5EBC50606EBF0
:1009400045153E4606EB85058E35984E96F90060B6
:10095000761EC6EBC60707EB4616954F07EB8606D5
:100960007668AA5D914D95F900506D1EC5EBC506E0
:1009700006EB45153E4606EB850569688B4D95F9F6
:1009800000506D1EC5EBC50606EB45153E4606EB51
:100990008505E868874D2D68A847844890F90000D0
:1009A000401EC0EBC00101EB4010814901EB80000B
:1009B00088307E4991F90010491EC1EBC10202EB5B
:1009C00041117B4A02EB81014968405C022842D117
:1009D000764890F90000401EC0EBC00101EB4010CA
:1009E000114601EB80002830704991F90010491E32
:1009F000C1EBC10202EB41116D4A02EB8101496872
:100A000010F8210040B2694908700B4693F9003094
:100A10005B1EC3EBC30505EB4313154605EB8303D0
:100A200003F14001614B93F900305B1EC3EBC3053A
:100A300005EB4313154605EB830358685B4B93F9AD
:100A400000305B1EC3EBC30505EB4313154605EBF6
:100A500083039A689047012C7ED1544890F9000096
:100A6000401EC0EBC00101EB4010514901EB80007A
:100A70000069002870D04D4890F90000401EC0EB7E
:100A8000C00101EB40104A4901EB8000002140F811
:100A90008E1F818047480068F0B3444D95F900509F
:100AA0006D1EC5EBC50606EB4515414E06EB8505EB
:100AB00040353E4E96F90060761EC6EBC60707EB42
:100AC00046163B4F07EB8606766855F82630374DBD
:100AD00095F900506D1EC5EBC50606EB45153E4663
:100AE00006EB85058E35314E96F90060761EC6EB15
:100AF000C60707EB46162E4F07EB86067668AA5DFB
:100B00002A4D95F900506D1EC5EBC50606EB45153F
:100B10003E4606EB850500E00FE06968234D95F938
:100B200000506D1EC5EBC50606EB45153E4606EBAF
:100B30008505E8681F4D2D68A8471C4890F90000FE
:100B4000401EC0EBC00101EB4010194901EB8000D1
:100B5000007C40B2154900E026E008700B4693F98E
:100B600000305B1EC3EBC30505EB4313104D05EBD3
:100B7000830303F140010D4B93F900305B1EC3EB7F
:100B8000C30505EB43130A4D05EB83035868074B78
:100B900093F900305B1EC3EBC30505EB4313044D13
:100BA00005EB83039A689047BDE8F081C9010020F6
:100BB00044110020D001002010B5044601F044F992
:100BC00001207649C86076488860002008610220CC
:100BD000886281F88800012081F88E00002048603A
:100BE0000220086002216D48C0F8A8106D49C0F8C5
:100BF000A4100021C0F8AC100321C0F8C4100221D9
:100C000080F824110421C0F8C810022180F82511B1
:100C10000521C0F8CC10022180F826110621C0F869
:100C2000D010022180F827110721C0F8D41002212A
:100C300080F828110021C0F8A01005205749C1F8FC
:100C40009C0003215548C0F844115749C0F8401191
:100C50000221C0F848110021C0F86011012180F87C
:100C6000C011002180F8C611C0F83C1100204B498A
:100C7000C1F8380107214948C0F8B4134B49C0F8FE
:100C8000B0130221C0F8B8130021C0F8D01300201F
:100C90004249C1F8A80304214048C0F8E011444982
:100CA000C0F8DC110221C0F8E4110021C0F8FC11E9
:100CB000012180F85C12002180F86212C0F8D8117E
:100CC00000203649C1F8D40105213448C0F87C120F
:100CD0003849C0F878120221C0F88012012180F84A
:100CE000F812002180F8FE12012180F8F91200218B
:100CF00080F8FF12012180F8FA12002180F8001319
:100D0000C0F8741203202549C1F870020621234857
:100D1000C0F818132849C0F814130221C0F81C1396
:100D2000012180F894130421C0F87C13012180F87C
:100D300095132021C0F88013012180F89613C82153
:100D4000C0F88413012180F897136FF00801C0F8F0
:100D500070131521C0F88813012180F89813C0F88A
:100D600070130721C0F88C130021C0F81013052060
:100D70000A49C1F80C0311480460114890F90000B9
:100D8000401EC0EBC00101EB4010044901EB8000A4
:100D9000002182680846904710BD000044110020E1
:100DA000990E010871180108F1160108F90D0108E2
:100DB00019140108051001089D140108D001002034
:100DC000C901002010B5054C44F82010183444F82F
:100DD0002020183444F8203010BD0000901400206A
:100DE0000149086070470000F001002001490870C7
:100DF00070470000EC010020F8B505460E46194882
:100E00000078062829D000F05FFF002404E0214686
:100E1000012000F0AAFF641C0C2CF8DD12A30122B3
:100E20004FF48171002001F00FF91148006811A3FF
:100E300002220A210090002001F006F90F480078F4
:100E40000FA303220A210090002001F0FDF80FA358
:100E500004220A21002001F0F7F806200149087059
:100E6000F8BD0000C8010020496E666F72000000E6
:100E7000F001002054503A2025730000EC010020BE
:100E80005645523A20562530327800004D443A20DB
:100E9000564F4C4C474F000070B504460D4619485C
:100EA000007800281ED018A30B220A21012000F090
:100EB00035FE002301221146184600F069FF18A3F1
:100EC00001225021002001F0BFF819A302225F2166
:100ED000002001F0B9F819A303225F21002001F0DE
:100EE000B3F80AE00CB9012100E00021084615A37F
:100EF000052240F2031101F0A7F800200149087013
:100F000070BD0000C8010020C9EEDBDACAD0CED621
:100F1000BDF8BFC6BCBCD3D0CFDEB9ABCBBE0000E2
:100F200056472D2D2D2D2D2D2D2D2D2D2D2D000008
:100F3000467265712E2A2A2A000000005077722E10
:100F40002A2A0000454E54455200000010B50446C0
:100F5000234601225021002001F076F810BD000048
:100F60002DE9FC4104462046FBF7DFFE8046084998
:100F7000FBF7BCFD0546FBF7FEFE06A30222CDE90A
:100F800000015021002001F05FF8BDE8FC81000065
:100F900000247449467265712E25362E32664D48FE
:100FA0007A0000002DE9FC4104462046FBF7BDFE17
:100FB00080460849FBF79AFD0546FBF7DCFE06A3D1
:100FC0000422CDE900015F21002001F03DF8BDE8D9
:100FD000FC81000000007A4442722E252E33666B9D
:100FE0006200000038B5044603A303225F210020FD
:100FF000009401F029F838BD5077722E25646442C0
:101000006D00000070B504460E46234800780428A1
:1010100017D000F059FE002504E02946012000F019
:10102000A4FE6D1C0C2DF8DD1CA301224FF4817170
:10103000002001F009F800F061F800F03DF800F040
:101040007FF804201449087008460078042821D14C
:101050000CB9012100E00021084613A302224FF43D
:10106000817100F0F1FF012C01D1012100E000218C
:1010700008460EA303224FF4817100F0E5FF022C15
:1010800001D1012100E00021084609A302227121BB
:1010900000F0DAFF70BD0000C8010020436F6E74DD
:1010A000696E756F75730000545800005258000047
:1010B00054585F4D440000002DE9FC410A48006887
:1010C000FBF733FE07460949FBF710FD0446FBF723
:1010D00052FE07A30322CDE9000140F203110020D4
:1010E00000F0B2FFBDE8FC81D801002000007A4486
:1010F00025372E33666B6270730000002DE9FC41CA
:101100000A480068FBF711FE07460949FBF7EEFCA9
:101110000446FBF730FE07A30222CDE900010521BA
:10112000002000F091FFBDE8FC810000E0010020FC
:101130000024744925362E32664D487A000000009E
:1011400008B5054890F9000004A30322052100908A
:10115000002000F079FF08BDE4010020256464420E
:101160006D0000007CB504460748007804280AD1C9
:101170002046FBF700FE05A30522CDE900010A2168
:10118000002000F061FF7CBDC80100207261746521
:101190003D25362E3266252500000000FEB50546A9
:1011A0000C460848007804280BD12846FBF7E3FDDD
:1011B00005A304228DE8130040F20311002000F083
:1011C00043FFFEBDC801002025352E3166252520B0
:1011D000253464007CB504460748007804280AD109
:1011E0002046FBF7C8FD05A30422CDE900010A2132
:1011F000002000F029FF7CBDC8010020433D2536BA
:101200002E32666D41000000F8B504460D460026FA
:101210000C480078042814D129462046FEF724FC07
:1012200009480AA3052212210090002000F00CFFBB
:101230000548143005A3062212210090002000F07A
:1012400003FFF8BDC801002088150020252D313589
:1012500073000000F8B504460D46002614480078D7
:10126000032823D113A305220A21002000F0ECFE5D
:10127000ADB117A305220A21002000F0E5FE00BF52
:101280000AE0207806F10C0213A30A210090002046
:1012900000F0DAFE641C761CAE42F2DB06E00FA31F
:1012A00005220A210020009400F0CEFEF8BD0000C7
:1012B000C8010020202020202020202020202020C5
:1012C000202020202020202020202020000000009E
:1012D0007061636B65743D00257800007061636B1D
:1012E00065743D252D3135730000000038B5044686
:1012F00006480078032807D105A303224FF4817123
:101300000020009400F0A0FE38BD0000C8010020BD
:10131000253036640000000038B504460B480078DC
:10132000032812D114F1960F0FDD0A2C0DDA42F2C8
:10133000107094FBF0F100FB114505A3022240F26E
:1013400003110020009500F07FFE38BDC801002089
:101350002530346464426D007CB50446074800784B
:1013600003280AD12046FBF706FD05A30222CDE99A
:1013700000010521002000F067FE7CBDC8010020AF
:10138000252D362E32666D4100000000F8B504466A
:101390000D4600261B480078032831D195B100BFC7
:1013A0000AE0207806F10A0117A305220090002028
:1013B00000F04AFE641C761CAE42F2DB2946204651
:1013C000FEF734FB29462046FEF730FB0F4810A3FA
:1013D000042212210090002000F036FE0B48143049
:1013E0000BA3052212210090002000F02DFE0748DB
:1013F000283007A3062212210090002000F024FECE
:10140000F8BD0000C80100202578000088150020E4
:10141000252D31357300000070B505460E4617487E
:101420000078032817D000F04FFC002404E0214688
:10143000012000F09AFC641C0C2CF8DD10A30122A2
:101440004FF48171002000F0FFFD10A3032205215D
:10145000002000F0F9FD03200849087008460078D4
:1014600003280AD10DB9012100E00021084609A393
:10147000062240F2031100F0E7FD70BDC801002014
:101480005061636B65742052580000005061636BBB
:1014900065743A0053544152540000002DE9FF474F
:1014A00004460E465B48007805282FD000F00CFC5F
:1014B000002504E02946012000F057FC6D1C0C2D8E
:1014C000F8DD55A301224FF48171002000F0BCFD2E
:1014D00053A302220A21002000F0B6FD52A30322EA
:1014E0000A21002000F0B0FD54A304220A210020AC
:1014F00000F0AAFD55A305220A21002000F0A4FD5A
:1015000056A306220A21002000F09EFD0520414935
:10151000087008460078052879D1554800680822E7
:1015200002EB820202F10A0100900CB9012200E0F4
:10153000002210464FA3022200F086FD4E480068AC
:10154000FBF7F3FB82464D49FBF7D0FA8146FBF7E8
:1015500012FCCDE902017068082202EB820202F15E
:101560000A010090012C01D1012200E00022104666
:1015700043A3032200F068FD44480068FBF7D5FB55
:1015800082463E49FBF7B2FA8146FBF7F4FB08229C
:1015900002EB8202CDE9000102F10A01022C01D125
:1015A000012200E00022104639A3042200F04CFD85
:1015B000394890F900000A22082302EBC301009089
:1015C000032C01D1012200E00022104633A30522A2
:1015D00000F03AFD33480068FBF7A7FB824632492A
:1015E000FBF784FA8146FBF7C6FB082202EB820276
:1015F000CDE9000102F10A01042C02D1012201E02F
:1016000005E00022104629A3062200F01DFDBDE8DA
:10161000FF870000C801002053657474696E67007D
:10162000547970653A00000043686E6C3A2D2D2D98
:101630002D2D2D2D2D2D2D4D487A000053746570C4
:101640003A2D2D2D2D4D487A000000005478506F12
:101650007765723A2D2D2D64426D000052664272FC
:101660003A2D2D2D2E2D2D2D6B6270730000000054
:10167000E801002025730000E001002000247449E7
:10168000253032642D3E25362E326600DC010020E6
:1016900025342E3266000000E4010020253033643A
:1016A00000000000D801002000007A4425372E33C6
:1016B000660000000149086070470000DC0100205E
:1016C0000149086070470000E001002001490860FE
:1016D00070470000D80100200149087070470000E1
:1016E000E40100200149086070470000E801002083
:1016F00070B505460E4617480078022817D000F04E
:10170000E3FA002404E02146012000F02EFB641CD3
:101710000C2CF8DD10A301224FF48171002000F0A1
:1017200093FC10A302220521002000F08DFC022072
:10173000084908700846007802280AD10DB901212D
:1017400000E00021084609A3062240F2031100F040
:101750007BFC70BDC80100205061636B6574205430
:10176000580000005061636B65743A005354415255
:101770005400000038B504460B480078022812D106
:1017800014F1960F0FDD0A2C0DDA42F2107094FB63
:10179000F0F100FB114505A3032240F203110020E4
:1017A000009500F051FC38BDC8010020253034649C
:1017B00064426D0010B5044605480078022805D142
:1017C000234603220A21002000F03EFC10BD000049
:1017D000C801002038B504460B480078022811D112
:1017E000601C38B909A3012240F20311002000F067
:1017F0002BFC07E007A3012240F203110020009414
:1018000000F022FC38BD0000C80100202020204F3D
:10181000555400002535646D730000002DE9FE432A
:1018200005460C460C480078022812D12846FBF7E2
:101830007CFA81460949FBF759F90646FBF79BFA02
:1018400007A302228DE8130040F20311002000F0EC
:10185000FBFBBDE8FE830000C80100200000204122
:1018600025352E31662525202020253564000000F1
:1018700070B504460E4600F027FA002504E029461C
:10188000012000F072FA6D1C0C2DF8DD01201C49BE
:1018900008700CB9012100E00021084619A30122BB
:1018A0000A2100F0D1FB012C01D1012100E000212F
:1018B000084619A302220A2100F0C6FB022C01D11E
:1018C000012100E00021084618A303220A2100F0AC
:1018D000BBFB032C01D1012100E00021084618A325
:1018E00004220A2100F0B0FB042C01D1012100E008
:1018F0000021084617A305220A2100F0A5FB70BDB0
:10190000C8010020456E74657220524620547261F1
:101910006E736D6974657200456E7465722052460F
:10192000205265636569766572000000456E7465D6
:101930007220524620436F6E74696E756F75730026
:10194000456E7465722052462053657474696E67E3
:1019500000000000456E7465722044657669636519
:1019600020496E666F7200002DE9F04106460C4674
:101970000D4FB046204604EBD0714910A4EB410155
:1019800009B1611C00E021468CB2002507E0384611
:10199000FCF7ADFA28F81500BF1C681C85B2A542FB
:1019A000F5DBBDE8F081000000E0030808B504485D
:1019B0000090022269460348FCF79CFA08BD00002B
:1019C000384B544100C0000870B505460C46264609
:1019D00004EBD6704010A4EB400008B1601C00E09E
:1019E000204682B229460248FCF784FA70BD000006
:1019F00000E003082DE9F0410746884614461848E0
:101A0000046040F6C410844202D9A4F6C41002E077
:101A100040F6C410001B054612480078E8B14FF0AC
:101A20007E5111480068FAF7D7FF0F490860C82DAA
:101A300007D24FF07E510D480068FAF7CDFF0B49F1
:101A400008600948016809480068FBF74FF8064636
:101A50000749FBF719F807490860BDE8F081000065
:101A600018000020080000201000002014000020B2
:101A70000000C8421C00002010B586B00446224871
:101A8000224908600846FCF709FD0220ADF8040071
:101A900048208DF8070002208DF8060001A91C4897
:101AA000FBF744FE01210220FCF7A4F81D208DF86D
:101AB000140000208DF8150001208DF816008DF817
:101AC000170005A8FCF726F80C20ADF80800022046
:101AD000ADF80A000120ADF80C000020ADF80E00B2
:101AE000ADF8100002A90B48FCF760FD0121094880
:101AF000FCF73BFD012210210648FCF7ADFD06482E
:101B0000046006B010BD0000152801085401002033
:101B1000000C014000040040400100202DE9F05F6E
:101B200081468A4693461E46002569E000244FF010
:101B3000010812E03548005D715D88420BD13349E0
:101B4000601C095C681C305C814204D14FF6FF7058
:101B500000EA041805E0A01C84B22C48005D7E2831
:101B6000E8DC00BFB8F1010F28D00223102259464B
:101B7000504600F0D4F800271BE0002415E0B9F12E
:101B8000010F07D1224911F80810C943C8B200F06B
:101B9000E7FA04E01E4911F8080000F0E1FA08F144
:101BA00001001FFA80F8601C84B2102CE7DB781C5F
:101BB00087B2022FE1DBA81C85B21DE002231022B0
:101BC0005946504600F0ABF8002711E000240BE026
:101BD000B9F1010F03D1FF2000F0C2FA02E00020AA
:101BE00000F0BEFA601C84B2102CF1DB781C87B2C6
:101BF000022FEBDB681C85B20AF1100000F0FF0A2F
:101C0000705D002892D1BDE8F09F0000512D0108C1
:101C1000722D01082DE9FF5F0C4615461E46002770
:101C2000AA4648E0F05D202843DBF05D7E2840DCDA
:101C3000F05D20381FFA80F90120C0EB4501022336
:101C40000822204600F06BF8A346AA464FF0000891
:101C500027E0B8F1080F02D10AF1010AA3460BF1FF
:101C6000010BBAF10C0F00DD1EE0BBF1C00F00DD6F
:101C70001AE00098012809D1124901EB091111F865
:101C80000810C943C8B200F06BFA06E00D4901EB39
:101C9000091111F8080000F063FA08F101001FFAB9
:101CA00080F8B8F1100FD4DB00BF0834C02C00DD81
:101CB00004E0781C87B2F05D0028B3DC00BFBDE80B
:101CC000FF9F0000722F010810B50C23C0220121D4
:101CD000084600F024F8002403E0002000F040FA59
:101CE000641CB4F5106FF8DB10BD0022002100BFAA
:101CF00006E0002201E0531C9AB20A2AFBDB491CD1
:101D00008142F6D3704710B50446302000F056F9F2
:101D1000F02000F011FA204600F022FA10BD2DE963
:101D2000F04104460D4616461F46641EED1D302048
:101D300000F044F9152000F0FFF9E0B200F010FACD
:101D4000A119491EC8B200F00BFA752000F0F4F991
:101D5000E8B200F005FAE919491EC8B200F000FA2D
:101D60005C2000F0E9F9BDE8F08170B505460E464B
:101D70000123082231462846FFF7D1FF002403E063
:101D8000FF2000F0EDF9641C042CF9DB70BD0000AD
:101D90002DE9F05F07460D4616461C46A946B24699
:101DA000284800EBC400B0F802B04FEAEB700BEB30
:101DB0005070C310234830F8342031462846FFF7CE
:101DC000AEFF4FF000082BE009F10109B9F1C00F97
:101DD00003DDA9460AF1010A20E0BAF10C0F00DD8B
:101DE0002DE0012F09D1174901EBC4014968097899
:101DF000C943C8B200F0B4F906E0124901EBC401CE
:101E00004968087800F0ACF90E4800EBC40040685F
:101E1000401C0C4901EBC401486000BF08F10108F7
:101E2000084931F83410074A02EBC402528801FB1A
:101E300002F0C11700EB5171B8EBE10FC4DB00BF3A
:101E4000BDE8F09F9C0F002008B51020ADF8000001
:101E50008DF8030003208DF8020069465448FBF713
:101E600065FC8020ADF8000010208DF803000320F1
:101E70008DF8020069464E48FBF758FC4020ADF84B
:101E8000000010208DF8030003208DF80200694641
:101E90004748FBF74BFC2020ADF8000010208DF8E0
:101EA000030003208DF8020069464148FBF73EFC21
:101EB000012210213E48FBF71FFD002220213C4853
:101EC000FBF71AFD6420FFF710FF0122202138489C
:101ED000FBF712FD42F21070FFF707FF302000F011
:101EE0006DF8942000F028F9312000F067F8D72031
:101EF00000F022F99F2000F033F9322000F01CF9A5
:101F0000002000F02DF9012000F02AF9032000F054
:101F100027F9302000F052F8082000F00DF9752064
:101F200000F00AF9002000F01BF9142000F018F965
:101F3000152000F001F9002000F012F9FF2000F058
:101F40000FF9BC2000F0F8F8002000F009F9A620F5
:101F500000F006F9CA2000F0EFF8002000F000F9C8
:101F60009F2000F0FDF8202000F0FAF81020FFF785
:101F7000CAFEFA2000F02EF8202000F0DDF80B2039
:101F800000F0EEF842F21070FFF7AFFEAF2000F065
:101F9000D3F842F21070FFF7A8FEFFF795FE054850
:101FA000054948605E2008804820488008BD000040
:101FB000000C0140023601089C0F002010B50446B9
:101FC00003480078A04202D0204600F0B5F810BDCA
:101FD000A301002010B50446C4F30804302000F02B
:101FE000ABF8812000F0A8F804F03F0000F0B8F84A
:101FF000A00900F0B5F810BD10B501224021074836
:10200000FBF77AFC012280210448FBF775FC0022D3
:1020100080210248FBF770FC10BD0000000C01405D
:1020200010B5012240210748FBF766FC0022802101
:102030000448FBF761FC012280210248FBF75CFCAD
:1020400010BD0000000C01400FB4F0B58FB0064683
:102050000C46174618A80E90342101A8FAF79DFCEB
:10206000322101A80E9B179AFCF740FD01A8FAF750
:102070009FFC0546C02D00DDC025B4F5817F06D14B
:1020800001A8FAF795FCC0004508C5F1600440F2CC
:102090000310844205D101A8FAF78AFCC500C5F1F6
:1020A000C00440F20110844200D1012401AB3A4641
:1020B00021463046FFF7AEFD00200E900FB0F0BC79
:1020C0005DF814FB70B50446002520E00022402195
:1020D0001848FBF711FC04F0800028B10122802190
:1020E0001448FBF709FC04E0002280211148FBF7AB
:1020F00003FC012240210F48FBF7FEFB0022402198
:102100000C48FBF7F9FB6006040E681CC5B2082DED
:10211000DCDB002280210748FBF7EEFB0122402197
:102120000448FBF7E9FB002240210248FBF7E4FBEF
:1021300070BD0000000C014010B504460748047053
:10214000FFF75AFF7820FFF7BDFF8020FFF7BAFFA7
:102150002046FFF7B7FFFFF763FF10BDA301002084
:1021600010B50446FFF748FF7820FFF7ABFFC0200B
:10217000FFF7A8FF2046FFF7A5FFFFF751FF10BDAF
:1021800070B50546002605E0601CC4B2C82C01DD10
:10219000002070BD02210E48FBF76CFE0028F3D032
:1021A00029460B48FBF772FE002405E0601CC4B210
:1021B000C82C01DD0020ECE701210548FBF75AFEA1
:1021C0000028F3D00248FBF75EFEC6B23046E0E7D7
:1021D0000030014010B50648006800B910BD00206D
:1021E000044908703620FBF795FF00BFF6E70000B2
:1021F00010020020140200200121014A11707047D2
:102200001602002010B586B0044601210803FBF732
:1022100001FDE020ADF8140018208DF81700032010
:102220008DF8160005A92348FBF780FA0020ADF8C9
:1022300000004FF48270ADF802000020ADF80400F9
:10224000ADF80600ADF808004FF40070ADF80A00D4
:102250001820ADF80C000020ADF80E000720ADF8F6
:10226000100069461448FBF713FE01211248FBF7E2
:10227000F5FD1020ADF814008DF8170003208DF83F
:10228000160005A90B48FBF751FA0220ADF814001F
:1022900048208DF8170003208DF8160005A907487F
:1022A000FBF744FAFBF78EF800F00CF804480460E2
:1022B00006B010BD0008014000300140000C014094
:1022C000180200201FB50220ADF8000003208DF891
:1022D000020048208DF8030069461748FBF726FAEC
:1022E0000220FBF7F7F80220019000208DF808008B
:1022F00008208DF8090001208DF80A0001A8FBF7DD
:1023000003F901210846FBF7F1F907208DF80C00CD
:1023100001208DF80D0000208DF80E0001208DF8B1
:102320000F0003A8FBF7F6FB0448054908600846C0
:10233000FBF7B8F81FBD0000000C0140052701089D
:102340001C02002070B505460C460748FFF75AFFEF
:10235000FBF75EFD3420FBF7DDFE0CB103480460A3
:10236000E5200349086070BDF92101080C02002036
:102370001002002010B5ADF50A7D2148006810B9A3
:102380000DF50A7D10BD1F48007800B9F8E7002060
:102390001C4908701C480078012802D002282BD163
:1023A0001AE020210DF22510FBF7FCFC3420FBF78E
:1023B000B1FE00201449087020208DF824014FF44C
:1023C000867247A96846FAF7CFFA00200F4C44A955
:1023D0000EC92468A04710E000200B4908704FF494
:1023E000867247A96846FAF7BFFA0320074C44A94A
:1023F0000EC92468A04700E000BF00BF00BFBFE7D0
:102400001002002016020020140200200C020020FE
:1024100010B50948006800B910BD012007490870CF
:102420003620FBF777FE3A20FBF774FE3420FBF7EB
:1024300071FE00BFF0E7000010020020140200202F
:102440000349096801B970470249086000BFFAE70B
:1024500010020020080200200149087070470000A7
:102460001502002070B504460D461B48006800B9EF
:1024700070BD00210846FFF765FF1848006800F0AE
:1024800031F824B1012C14D0022C21D110E0042009
:102490001349087033211220FCF712FB3620FBF79A
:1024A00039FE3B20FBF736FE3520FBF733FE10E00C
:1024B0000FE003200A49087035210820FCF700FBD3
:1024C0000D210220FCF7FCFA3420FBF723FE00E08C
:1024D00000BF00BF00BFCBE71002002004020020B5
:1024E0001402002010B504460548006800B910BD6C
:1024F0000448046001780A20FCF7E2FA00BFF6E71E
:1025000010020020040200200349096801B9704745
:102510000249087000BFFAE7100200200002002004
:1025200010B504460648006800B910BD02200549F0
:102530000870217B04F10D00FBF764FD00BFF4E798
:1025400010020020140200207FB505460C461948F1
:10255000194908600846FBF759FF0121C802FBF73B
:1025600059FB19208DF8000000208DF801008DF82E
:10257000020001208DF803006846FBF7CBFAA8B2F1
:10258000ADF808004720ADF804000020ADF80A00BF
:10259000ADF8060001A90948FCF794F8012211469C
:1025A0000648FCF759F801210448FBF7DEFF044810
:1025B00004607FBDFD270108AC010020002C014014
:1025C000A801002030B587B005460C462A482B49A3
:1025D00008600846FCF730F901218803FBF71AFB75
:1025E0004FF40070ADF8180003208DF81A00182081
:1025F0008DF81B0006A92248FBF798F84FF480607D
:10260000ADF8180004208DF81B0006A91C48FBF744
:102610008DF825208DF8040003208DF805008DF835
:10262000060001208DF8070001A8FBF773FA029558
:102630000020ADF80C00ADF80E00ADF81000ADF8BC
:1026400014000C20ADF8120002A90E48FCF7A0F906
:10265000012240F225510B48FCF775F9012240F2A6
:1026600024410848FCF76FF901210648FCF728F9D6
:102670000548046007B030BDC128010824010020CE
:1026800000080140003801401C01002070B50446DC
:102690000D4603E0207800F007F8641C281EA5F121
:1026A00001018DB2F6D170BD10B5044600BF4021C6
:1026B0000448FCF711F90028F9D021460148FCF73D
:1026C000D8F910BD0038014010B501210420FBF7F6
:1026D000A1FA01210820FBF79DFA01211020FBF748
:1026E00099FA01212020FBF795FA01210803FBF755
:1026F00091FA01210846FBF78DFA4FF48040FBF771
:102700006DFA10BD70B504460D460448006818B156
:10271000012002490968884770BD000018020020A6
:102720000FB410B504464FF48C7203A91A48FAF797
:102730001BF934B1012C1CD0022C1ED0032C25D146
:102740001FE0FFF765FE0A20FDF7B2F81348007896
:1027500070B1032212A110481530FAF730F938B9D8
:102760004FF07E510F480068FAF736F90D490860BE
:102770000DE00E20FDF79CF809E00E20FDF798F81B
:1027800005E0FBF74DF9FFF743FE00E000BF00BF97
:1027900010BC5DF814FB0000280400200800002095
:1027A00068656C001400002070B504460E4615469E
:1027B0000120FCF7C0F904EB44000E4901EB800056
:1027C0008560002004EB44010A4A02EB8101486065
:1027D00004EB4400114601F8206035B90120A04007
:1027E000054909680843044908600020FCF7A3F97B
:1027F00070BD0000C40F0020BC01002070B504466D
:102800000D460348006810B101480068804770BD5C
:10281000A801002070B504460D462148008840B943
:102820002048FBF7AEFE2049088001201C490880A3
:1028300034E01B480088012830D11A48FBF7A1FE7C
:102840001A4908800846008817490988884207DD28
:102850001648008814490988401A1549086009E09B
:10286000114800884FF6FF71081A1049098808447A
:102870000F4908600F4800680D490968B0FBF1F086
:102880000D4908600020064908800B480268074887
:10289000018805480088094B1B68984770BD0000F7
:1028A00034010020000400403001002032010020EB
:1028B00038010020080100203C01002040010020D8
:1028C00070B504460D4614B1012C1ED10DE0104820
:1028D00001881048104A12689047FF210D48FAF706
:1028E0005CF800200A49088010E00A48084A12886B
:1028F000855407480088401C054908800846008820
:10290000FE2801DD0020088000E000BF00BF70BD90
:10291000200100206F0600201C0100202DE9F0415D
:1029200007460D4614461E46781E06287DD2DFE86F
:1029300000F07C032B51046828E125B1012D10D053
:10294000022D1ED115E00CB1052100E0062108463C
:10295000FCF7AEFF0CB1042000E000208D490870A8
:1029600010E00CB1062100E007210846FCF7A0FFAB
:1029700008E00CB1082100E007210846FCF798FFA9
:1029800000E000BF00BF01E115B1012D1ED11EE026
:1029900014B14FF4FA7300E000231A460CB101237E
:1029A00000E0002319460CB10B2300E00723184672
:1029B000FFF7FAFE0CB1022000E000207549087014
:1029C0000020754908607549086001E000BF00BF3C
:1029D00000BFDBE095B90CB10C2100E007210846EF
:1029E000FCF766FF0CB1032000E000206949087085
:1029F0000020694908606949086000E000BF00BF25
:102A0000C4E0052D7DD2DFE805F0034A6B99AF00E5
:102A100063490E770846C17E072302220420FEF791
:102A2000D1F95F4991F91A0000E0AEE0FFF76CFDC3
:102A30005B4991F91A105B4A5056FEF74DFE584912
:102A4000C97E594A52F82100FEF740FE5449097FD9
:102A500001EB8101554A02EB8100FEF743FE50492C
:102A6000097E4F4A527E11FB02F101EB81014900C0
:102A700001EB4102C2EBC111494A127F4C4B53F8A2
:102A8000222002EBC100FEF71BFE4549087EFFF73E
:102A900029FDC82200210920FFF786FE73E0404986
:102AA0000E76097E3E4A527E11FB02F101EB810156
:102AB000490001EB4102C2EBC111394A127F3C4B84
:102AC00053F8222002EBC100FEF7FAFD3449087EDC
:102AD000FFF708FDC82200210920FFF765FE52E03C
:102AE0002F494E76497E01EB810149004FF47A72FD
:102AF00011FB02F0FEF7DEFD2949097E284A527ECD
:102B000000E03FE011FB02F101EB8101490001EB24
:102B10004102C2EBC111224A127F254B53F82220F9
:102B200002EBC100FEF7CCFD1D49087EFFF7DAFC81
:102B3000C82200210920FFF737FE24E070B21849AF
:102B4000887691F91A10174A5056FFF7DDFC1449A0
:102B500091F91A10134A5056FEF7BEFDC822002103
:102B60000920FFF721FE0EE00D49CE76C97E0E4A00
:102B700052F82100FEF7AAFDC82200210920FFF724
:102B800013FE00E000BF00BF00E000BF00BFBDE8D3
:102B9000F0810000350000202000002024000020EB
:102BA00050060020482D01082C2D01083600002079
:102BB0001C2D010810B5574890F90000401EC0EBCD
:102BC000C00101EB4010544901EB80008E305149A7
:102BD00091F90010491EC1EBC10202EB41114E4AAE
:102BE00002EB81014968405C002875D0494890F9A2
:102BF0000000401EC0EBC00101EB4010114601EB8C
:102C000080009430434991F90010491EC1EBC10284
:102C100002EB4111404A02EB81014968405C08B96E
:102C2000012200E000223B4890F90000401EC0EB6A
:102C3000C00101EB4010384901EB80019431354867
:102C400090F90000401EC0EBC00303EB4010324B74
:102C500003EB800040680A542E4890F90000401EA3
:102C6000C0EBC00101EB4010194601EB800094302D
:102C7000284991F90010491EC1EBC10202EB411134
:102C80001A4602EB81014968405C30B3214B93F94D
:102C900000305B1EC3EBC30404EB4313144604EB88
:102CA000830303F140011B4B93F900305B1EC3EB20
:102CB000C30404EB4313144604EB83035868154B19
:102CC00093F900305B1EC3EBC30404EB43131446BB
:102CD00004EB83039A6890471BE00E4890F90000CC
:102CE000401EC0EBC00303EB40100B4B03EB800016
:102CF00000F14001074890F90000401EC0EBC003FE
:102D000003EB4010044B03EB800082684FF0FF3070
:102D1000904710BDC901002044110020400ECF197A
:102D200080CE341D00A1BC33C0CA89368813000090
:102D30008813000088130000881300008813000027
:102D40008813000088130000E2ECF1F60600050786
:102D50000AC9EEDBDACAD0CED6BDF8BFC6BCBCD33A
:102D6000D0CFDEB9ABCBBEA1FAA1FBA1FCA1FDA1E6
:102D7000E800080640310070444850435048447011
:102D8000000020207E8004848890A0FFA09088848A
:102D90000400040404FF040400FF00007F0000FF9F
:102DA0000000080C08F0101106F80000FC0000FFFD
:102DB0000000001011111111915F1111111111106A
:102DC00000000000FC00000000FF00000804F80004
:102DD00000000806403100212121217F41C141012D
:102DE000010020207E800102041860806018040227
:102DF00001000202423300011111FF1111FF1111F4
:102E00000100000204F804020A32C20202FA0202BD
:102E100002002424257FC5440044330000FF000045
:102E20000000106080FF00802020202020FF404014
:102E30004000080808FF080910111111FF111111B5
:102E40001000202241FE80010102C2340814628178
:102E5000010020202021273CE424242424272020B2
:102E6000200020408000FF909090909291FE000002
:102E70000000007F445A61007F49494949497F0069
:102E8000000000FF2010E000FF0204C03028448250
:102E900002000001020418600100E01804020100B1
:102EA00000008000040E1464840404241C060080C6
:102EB00080000008484949494949494848407F003D
:102EC0000000000000FC08080808FC000201FE00E9
:102ED00000000101010101010101090507030301CE
:102EE000010000000000000000002040C0808000C1
:102EF00000000101030307050901010101010101AE
:102F0000010000008080C0402000000000000000A0
:102F1000000000000000020C38FF380C0200000026
:102F2000000000000000000000FF000000000000A2
:102F3000000000000000000000FF00000000000092
:102F400000000000000040301CFF1C30400000006A
:102F50000000004020170810101010101008172053
:102F60004000000204E81008080808080810E804F7
:102F7000020000000000000000000000000000004F
:102F800000000000001F00000000000000CC000056
:102F90000000000830400830400000000000000041
:102FA00000000002031E02031E000020FC2020FC83
:102FB0002000000E11113F100C0000180404FF84C3
:102FC00078000F100F0106180000008C30C07884C4
:102FD0007800000F10110E0000007884C43498E4CB
:102FE000840800487000000000000000000000009D
:102FF00000000000000718204000000000E0180456
:103000000200004020180700000000020418E00041
:1030100000000202010F01020200404080F08040E7
:103020004000000000000700000000808080F08069
:103030008080000000000000000000090E00000079
:103040000000000000000000000000808080808000
:1030500080000000000000000000000C0C000000D8
:10306000000000000000031C2000000618E0000023
:103070000000000708101008070000F0080404080A
:10308000F000000008081F00000000000404FC0419
:103090000400000E101010100F00000C14244484C3
:1030A0000C00000C101010110E0000180484844451
:1030B0003800000001020C1F00000060A02424FC66
:1030C0002424001F1111111010000098040404881A
:1030D0007000000708111109000000F088040404C2
:1030E000F80000181010111618000000007C800075
:1030F0000000000E111010110E00003844848444AA
:103100003800000F10101008070000804844448861
:10311000F00000000003030000000000000C0C00A1
:103120000000000000010000000000000007000097
:103130000000000001020408100000804020100878
:10314000040000020202020202000040404040402F
:103150004000001008040201000000040810204094
:103160008000000E121010110E000000000CEC0088
:103170000000030C131417080700E018E414F414FB
:10318000E8000000031C07000000043CC44040E4C9
:103190001C04101F1111110E000004FC040404880B
:1031A0007000030C101010101C00E0180404040838
:1031B0001000101F10101008070004FC040404087D
:1031C000F000101F11111710080004FC0404C404BF
:1031D0001800101F11111710080004FC0400C00093
:1031E0000000030C1010101C0000E01804044478C8
:1031F0004000101F100000101F1004FC8480808409
:10320000FC040010101F10100000000404FC040453
:103210000000000010101F10100003010101FE004B
:103220000000101F11031418100004FC0480641C1B
:103230000400101F10000000000004FC040404043B
:103240000C00101F1F001F1F100004FC807C80FC5E
:103250000400101F0C0300101F1004FC0400E018F1
:10326000FC000708101010080700F0080404040808
:10327000F000101F101010100F0004FC84808080DC
:1032800000000708101010080700F00814140C0ABA
:10329000F200101F111111110E0004FC0400C030C7
:1032A0000C04000E111010101C00001C0484844437
:1032B00038001810101F10101800000004FC040043
:1032C0000000101F100000101F1000F80404040478
:1032D000F800101E110000131C100000E01C70808C
:1032E0000000101F001F001F100000C07C807CC069
:1032F00000001018160101161810040C34C0C03458
:103300000C04101C1300131C1000000004FC04002B
:10331000000008101010131C1000041C6484040426
:1033200018000000007F40404000000000FE020244
:10333000020000201C030000000000000080601C50
:103340000300004040407F00000000020202FE0037
:1033500000000000204040200000000000000000AD
:103360000000000000000000000001010101010157
:1033700001010040402000000000000000000000AB
:10338000000000000101010000000098242448FC16
:103390000400080F00010100000000FC88040488FC
:1033A00070000000000101010000007088040404A6
:1033B00088000000010101090F0000F8040404085E
:1033C000FC04000001010101000000F82424242471
:1033D000E8000001010709090400000404FC0404DA
:1033E0000000000001010101010000D6292929C9BE
:1033F0000600080F00010101000004FC8400000425
:10340000FC040001191900000000000404FC04047D
:10341000000000000001191900000003010101FE75
:103420000000080F00000101010004FC2460940C5E
:1034300004000008081F00000000000404FC04044D
:103440000000010101010101010004FC0400FC0471
:1034500000FC010100010101000004FC84000004E3
:10346000FC04000001010101000000F80404040450
:10347000F800010100010100000001FF8904048837
:103480007000000000010100010000708804048940
:10349000FF0101010100010101000404FC8404009A
:1034A0008000000001010101010000CC242424243B
:1034B00098000001010701010000000000F8040469
:1034C0000800010100000001010000F804040408E4
:1034D000FC04010101000101010000C0300C30C0FA
:1034E0000000010100010100010180700C30E01CAE
:1034F0006080000101010001010000048C70748CE7
:10350000040001010100000101010081611E186039
:103510008000000101010101010000840C34448499
:103520000C0000000000003F404000000000807CD4
:10353000020200000000FF00000000000000FF0089
:10354000000040403F000000000002027C800000BC
:1035500000000040804040204000000000000000CB
:103560000000F8F80CC40CF8F00003070C080C0776
:103570000300001018FCFC0000000008080F0F08F2
:103580000800080C84C4643C18000E0F0908080CDD
:103590000C00080C444444FCB800040C0808080F54
:1035A0000700C0E0B098FCFC8000000000080F0F8E
:1035B00008007C7C444444C48400040C0808080FC0
:1035C0000700F0F84C4444C08000070F0808080FBB
:1035D00007000C0C0484C47C3C0000000F0F0000AA
:1035E0000000B8FC444444FCB800070F0808080F6A
:1035F0000700387C444444FCF800000808080C0725
:1036000003000000000000000000000000000000B7
:1036100000000000000000000000000000000000AA
:1036200000000000000000000000000F1F3F7F7F2F
:103630007FFF7F7F7F3F1F0700000000000000002A
:10364000000000000000000000000000000000007A
:10365000000000000000000000000000000000006A
:10366000000000000000000000000000000000005A
:103670000000000000000000000000000000010148
:10368000010101010100000000C0E0F0F8F8FCFCBD
:10369000FCF8F8F0E08000000101010101010100E7
:1036A000000000000000000000000000000000001A
:1036B000000000000000000000000000000000000A
:1036C00000000000000000000000000000000000FA
:1036D0000000000000000000003F7FFFFFFFFFFF31
:1036E000FFFFFFFF7F1E0000000000000000000041
:1036F0000000003F7FFFFFFFFFFFFFFFFFFF7F1E78
:1037000000000000000000000000000000000000B9
:1037100000000000000000000000000000000000A9
:103720000000000000000000000000000307070F79
:103730000F0F0F0F0703010080C0E0E0F0F0F0E092
:10374000F0F8FC7E3F1F0F070F0F0F0F0F0F1F3FEB
:103750007EFCF8F0E0E0F0F0F0E0E0C08000000077
:103760000307070F0F0F0F0F0703010000000000F2
:103770000000000000000000000000000000000049
:10378000000000000000000000F8FEFFFFFFFFFF48
:10379000FFFFFFFFFFF90100000000000000000034
:1037A0000000F8FEFFFFFFFFFFFFFFFFFEFCF80039
:1037B00000000000000000000000010103FFFFFF07
:1037C000FFFFFFFFFFFFFFFEFCF80000000000000E
:1037D0000000000000000000010F1F3F3F3F7F7FFF
:1037E0003F3F3F1F0F01000000000080808080806D
:1037F000C0E0F0F8FFFF7F3F3F7F7F7F3F3F1F0F1D
:1038000003000000808080808000000000070F1F00
:103810003F3F7F7F7F3F3F7FFFF3E0C0800000801E
:103820008080808000000000010F1F3F3F3F7F7FAE
:103830003F3F3F1F0F0180E0F8F8FCFCFCFCFCFC64
:10384000FCFEFF8F0F0703010101010101010101CE
:103850000307EFFFFFFEFCFCFCFCFEFFFFFFC703BE
:103860000301000101010101010307EFFFFFFEFC5D
:10387000FCFCFCFCFCFEFFDF0F0703030101010160
:10388000010103070F1FBFFEFCFCFCFCFCFCFCFC61
:10389000F8F8E080000000000000000000000000D8
:1038A0000080C0FFFFFFFFFFFFFFFFFFFFFFFFDE06
:1038B000800000000000000000000080C0FFFFFF4B
:1038C000FFFFFFFFFFFFFFFFFFDE800000000000A3
:1038D00000000000000080FFFFFFFFFFFFFFFFFF71
:1038E000FFFFFF9E0000000000000000000000003D
:1038F00000000000000000000000000000000000C8
:103900000000C0C0E0F0F0F0F0E0E0C08000000097
:10391000000000000000000000000000C0C0E0F057
:10392000F0F0F0E0E0C080000000000000000000C7
:10393000000000000000C0C0E0F0F0F0F0E0E0C0E7
:1039400080000000000000000000000000000000F7
:103950000206034708050B060D100EA70F6210C7DD
:10396000118312131540181819161B4320FB23E965
:10397000242A2500261F2C812D352E099C3901086B
:103980000000002024020000BED100080C3A01080B
:1039900024020020A417000028EB000801122B804D
:1039A0003F047A010CA183B80BC80F56473232315D
:1039B00032533433334E30533114FB393014FC3826
:1039C000363814AC393135145C3131300C813982E0
:1039D00004671408027CA24A047A00084402030423
:1039E00006070809294C6950051002040608130D42
:1039F000DA1408F9D9B9181A6D141A5904193E19AC
:0C3A00000201260A26FF2931022FC00017
:040000050800C931F5
:00000001FF
